:10000000F0230010219000001F9000001F900000BE
:100010001F9000001F9000001F90000000000000D3
:100020000000000000000000000000001F90000021
:100030001F900000000000001F900000718600006B
:10004000818400008184000081840000818400009C
:10005000818400008184000081840000818400008C
:10006000818400008184000081840000818400007C
:10007000818400001D9000001D900000018D000093
:100080000D870000258700003D8700005587000090
:100090001D9000006D8700001D9000001D90000065
:1000A0001D9000001D9000001D9000001D9000009C
:1000B0001D9000001D9000001D9000001D9000008C
:1000C0000523F0B520385843344B87B01B78002502
:1000D0000293334B1B789C46842353430493314B48
:1000E000C3180593059B029A5B5D0800009393403B
:1000F0000022DBB2019262465218D2B2904247D03F
:10010000049A8418284AA2180392002434E00100BB
:10011000E8E76646022E18D1009FA3001F413B006E
:100120000D3633409F001F4333231F407B003B436A
:10013000463633405F003B435B00DBB2002A21D0F0
:10014000019A002A01D001221343552216005F08AC
:1001500017405A00B2431743FFB2223EBA08BF000D
:10016000B74332403A438427D2B26743160912019B
:100170003243039E0134F255E2B29445C9D80130AE
:10018000C0B2B8E75AB2002ADFDA01220192DCE7F6
:100190000135052DBBD107B0F0BDC046610600108A
:1001A0001B00001074BE000020120010F8B50400FF
:1001B0000D00160006272078002800D1F8BD290080
:1001C0003200FFF77DFF034B0134197879436D1836
:1001D000EDB2F0E71B0000108423CA08534318183F
:1001E000842310B55B00984208DA0722083B8A4353
:1001F000FF3B9340024C225C1343235410BDC04686
:100200002012001070B5114B01201B78002B1BD061
:100210000F4A013B1B01D3189D68DC6800220023B4
:100220002800210009F0B2F8002802D080231B0624
:10023000E418084A084B2800210009F0BBF8030025
:1002400001205A1E9341584070BDC046DC05001085
:10025000E00500103EC3D84E7D7F612B7047000043
:100260000023034A1370034A1370034A1370704744
:10027000DA05001095060010DB050010024A13781D
:1002800059424B4113707047890600100023044AFD
:100290001370044A13700122034B1A707047C04652
:1002A00093060010920600108C0600100023044AEA
:1002B0001370044A13700222034B1A707047C04631
:1002C00093060010920600108C0600100023034ACB
:1002D0001370034A1370034A13707047930600109B
:1002E000920600108C060010024A137859424B41C6
:1002F00013707047910600100122034B1A70002200
:10030000024B1A707047C046920600108C0600100F
:100310000122034B1A700022024B1A707047C0462C
:10032000930600108C0600100122014B1A707047D2
:10033000980600100849094A0B78002B05D0107860
:10034000074B1B18FF20013B1870002301200B7086
:100350000449137008707047A10600105808001077
:100360003B00001099060010024A137859424B4195
:10037000137070479D0600100222034B1A70002272
:10038000024B1A707047C0469D0600108C06001084
:100390000322034B1A700022024B1A707047C046AA
:1003A0009D0600108C0600100022014B1A70704749
:1003B0009A0600100022034B1A70034B01321A7088
:1003C0007047C04658080010A106001000230F4ACD
:1003D00070B513700E4A10241370002300220D4EC6
:1003E0000D4930000A604B608A60CB60220008F043
:1003F000DDFB0A4D31002200280008F0D7FB290060
:100400002200074808F0D2FB70BDC046DC05001092
:1004100038130010701300108013001060130010C8
:10042000501300100122034B1A700022024B1A7065
:100430007047C046200000108C0600100023024ABE
:100440001370024A13707047200000108C060010D1
:100450000122014B1A707047A50600100122014BC2
:100460001A7070479706001010B5021C202800D99A
:100470002022002003000649D2B2934200D310BDCF
:100480000C5CFF2C01D10133DBB20130F5E7C04633
:100490005F08001070B5074B1D78681CC0B2FFF7ED
:1004A000E3FF04002800FFF7DFFF013C201AC0B281
:1004B00070BDC0462813001010B5FFF7D5FF034BE1
:1004C000185CFE3843425841C0B210BD5F080010AE
:1004D000034B1A78034B1A700022034B1A707047B3
:1004E0008A060010890600109F06001010B50A4BFE
:1004F0001878FFF7B9FF0023084A12180848D45C9F
:10050000D9B2FF2C02D0242B03D11900FF2343546E
:1005100010BDC4540133F2E7281300105F08001027
:1005200034080010074A002013780021002B07D060
:10053000013BDBB21370044ADB00D318186859681A
:100540007047C04693190010981900100023034A01
:100550001370034A1370034A13707047AA06001001
:100560009119001092190010044A137859424B4116
:1005700013700022024B1A707047C0462100001011
:1005800091060010054B1A78002A02D000221A703A
:10059000704701211970024BF9E7C046910600101F
:1005A000210000100022014B1A707047A9060010AC
:1005B00002000020030010B5074C934204D2215CD6
:1005C000002901D0FF2800D110BD0130C0B20A2996
:1005D000F3D10133DBB2F0E7850000100023054AB8
:1005E000D15C581C002901D0FF2B01D1C0B270474B
:1005F000C3B2F5E785000010002318000649CA5C65
:10060000002A01D0FF2B00D170470133DBB20A2A48
:10061000F5D10130C0B2F2E785000010084B400070
:1006200070B5C45C1B185D7820002900002207F01B
:100630002DFE29000122200007F074FE70BDC04687
:10064000B4C200000122F8B508210600100007F02E
:1006500069FE0724082700223900012007F062FE06
:10066000320001252241022100202A4007F05AFED3
:100670002A003900280007F055FE013CEBD2F8BDF6
:10068000002210B504001100022007F04BFE2000EC
:10069000FFF7D8FF10BD0000A022FF21520010B5C7
:1006A000094808F0A4FA202300200021074A013B52
:1006B000DBB203C2002BFAD1054A1370054A13704E
:1006C000054A137010BDC0465F08001020110010CD
:1006D000281300102A13001029130010F8B5551C18
:1006E00086180C001700451908F0B9FAC21B310032
:1006F0002800013208F09DFA3470F8BD30B50E4C78
:1007000085B0039323780D4D009001910292072B41
:1007100007D9702228000A4908F08BFA2378013B98
:10072000237020781022431C00016946281823708A
:1007300008F03CFA05B030BDDC050010E005001003
:10074000F005001010B50B4B197800290BD00A4C9E
:100750000A4B0139090110222000591808F026FA25
:100760000FCCFFF7CBFF0023054A1370054A137027
:1007700010BDC046DC050010B0060010E0050010FA
:10078000DB050010DA05001010B5FFF7DBFFFFF7FF
:10079000D9FF0122034B1A700023034A1370034A46
:1007A000137010BDA7060010AD0600101F11001039
:1007B00030B5002204000D00002385B0009401959F
:1007C00002920393009801990022039BFFF796FF82
:1007D0002000290005B030BDC02010B50249C00579
:1007E000FFF7E6FF10BDC046FB210940802110B590
:1007F0000020C905FFF7DCFF10BD00001FB5002277
:1008000000230092019300220020054B01990292DF
:100810000393039B0200FFF771FF05B000BDC046C4
:100820000000F03F10B5024B0FCBFFF767FF10BD84
:10083000B006001010B5024B0FCBFFF75FFF10BDE5
:1008400040130010F8B5070020200E001400FFF739
:100850000BFEA02305005B0098420BD23800FFF787
:1008600003FE24182A1B044D601C6119401908F06E
:10087000E0F92E55F8BDC0465F080010F8B5060037
:100880000120FFF7F1FD471E04002020FFF7ECFDDB
:10089000054D0130021B7919601908F0CAF90022D0
:1008A000024BEE551A70F8BD5F0800108E0600105E
:1008B000F8B50C4F06003B780D000B4C032B08D904
:1008C000210018222000083108F0B3F93B78013BE1
:1008D0003B703B785A1CDB00E4183A702660656078
:1008E000F8BDC046931900109819001010B5094BB7
:1008F0001B78002B07D0084A013BDB00D31818688F
:100900005968FFF7D5FF0023044A1370044A137097
:1009100010BDC0469319001098190010AA060010C7
:100920009219001010B5FFF7FDFD002342428B41E4
:1009300010001900FFF7BCFF10BD000070B5FFF7F5
:10094000F1FD05000C00FFF7EDFD074B1B78002BB8
:1009500003D06422002308F065FD2A00230008F07C
:100960003DFDFFF7A5FF70BD2100001070B5FFF73A
:10097000D9FD0D000400FFF7D5FD00196941FFF70F
:1009800097FF70BD10B5FFF7CDFFFFF7EFFF10BD6C
:1009900070B5FFF7C7FD05000C00FFF7C3FD284049
:1009A0002140C043C943FFF783FF70BDF8B5040081
:1009B0000025074E8322330083331F78310005481A
:1009C000013508F036F93770A542F2D1F8BDC046BE
:1009D0002012001021120010F8B5040008F03FF9B1
:1009E0000023C7B2661EDAB2E118BA4203D25A1C1B
:1009F000B55C202D06D0C2B2D21A2000013208F018
:100A0000D5F8F8BD1300EEE770B5851808000C00A6
:100A100008F025F921000200280008F0C7F870BD91
:100A2000F0B5002489B003221A49019004AF03A84D
:100A30003C7108F0BBF80622174906A808F0B6F882
:100A4000E5B20321280008F015FB144BC6B21E7056
:100A5000019BA10059180422380008F0A7F82800CB
:100A6000032108F08DFB03ABC9B25D5C06ABE05C13
:100A7000290080383200C0B20635FFF721FB01346F
:100A800032003800E9B2FFF791FB062CD8D109B04B
:100A9000F0BDC04678BA00007CBA000061060010C4
:100AA00070B5C2000400002100200E4B9B18186096
:100AB00059602000FFF7D8FC0B4E0500335CFF2B7C
:100AC0000ED00134E0B2FFF7CFFC04002020FFF786
:100AD000CBFC611E0130021B8919A81908F066F8C9
:100AE00070BDC046201100105F08001010B50C004A
:100AF000FFF7BAFC24182020FFF7B6FC021B0348BE
:100B0000611C0918201808F051F810BD5F0800108A
:100B1000F8B505000026064C8322277820000549F9
:100B20008334013608F042F82770AE42F3D1F8BDA5
:100B30002012001021120010F8B5124B1F78781CFB
:100B4000C0B2FFF735FD104D041E104E0CD10A2324
:100B500030702B706870300008F081F801220C4B67
:100B600018700C4B1A70F8BD3800FFF721FD241ADD
:100B7000013C29182200300008F018F800233355F2
:100B8000E9E7C046901300108500001063060010CE
:100B9000620600108F06001010B58424C2B06400F5
:100BA00022006846044908F001F82200694603481B
:100BB00007F0FCFF42B010BD80BB00002012001007
:100BC000F7B516001F0002000B00009001913000E5
:100BD000390009F023FB04F067FD0022154B09F0F2
:100BE0001FFFC022144BD20509F018FB002204009D
:100BF0000D0000980199002308F0C8FB00280FD0D1
:100C0000002200233000390008F0C0FB0022094B0D
:100C1000002809D0200029000AF06EF904000D0018
:100C20002000290003B0F0BD2000290008F0BAFF21
:100C3000F4E7C04600806640FB21094013B507F089
:100C40001BF901A9684607F0BFF96B46587908F00F
:100C50005BFF084908F040FE6B46041C187908F059
:100C600053FF011C201C08F099FC0AF081FDFFF7DE
:100C70009FFD13BD0000C84210B507F065F808F0ED
:100C800043FF044908F028FE0AF072FDFFF790FDCB
:100C900010BDC04600007A440023F7B5114F124D35
:100CA0003B702B70984218D1104B01241878FFF735
:100CB000DBFB0F4E3618335DFF2B0AD06A461371EB
:100CC00000232800537101A901340AF0AFFE082C5B
:100CD000F1D1280007F0C3FF38700122054B1A70CC
:100CE000F7BDC0466206001063060010281300100E
:100CF0005F0800108F06001010B50B49040000209B
:100D0000002C0CDC013464B2012C0CD00022074B07
:100D100009F084FAF6E70022044B09F081FE013C59
:100D200064B2631CF7D110BD0000F03F0000244006
:100D300010B50B4B0400197800290AD00139C9B24B
:100D40001970084B09011022591807F02FFF2000D5
:100D500010BD00220023026043608260C360F6E79A
:100D6000DC050010E005001000B58DB06846FFF707
:100D7000DFFF04A8FFF7DCFF009A019B04980599A8
:100D800008F010FF029A039B0890099106980799B2
:100D900008F008FF0A900B910A9A089809990B9B92
:100DA000FFF7ACFC0DB000BD10B500200249FFF705
:100DB000FFFCFFF7D9FF10BD0000F03FF0B589B090
:100DC0006846FFF7B5FF009C019D029E039F22002D
:100DD0002B003000390009F021FA32003B0009F005
:100DE0001FFE22002B0008F0DDFE02000B00002099
:100DF000114909F013FA3200049005913B002000DC
:100E0000290009F00BFA22002B0009F009FE32003C
:100E10003B0008F0C7FE02000B000020074909F064
:100E2000FDF906900791069A04980599079BFFF72C
:100E300065FC09B0F0BDC0460000F03F0000F0BF07
:100E4000F0B593B006A8FFF773FF069B079C0AA8AE
:100E500000930194089C099DFFF76AFF0A9E0B9F6F
:100E60000C9A0D9B009801990292039332003B006B
:100E700009F0D6FD029A039B0490059120002900F9
:100E800009F0CEFD02000B00049805990AF034F831
:100E900032000E900F913B002000290009F0C0FDA8
:100EA000029A039B04000D000098019909F0B8FD17
:100EB00002000B002000290008F074FE1090119130
:100EC000109A0E980F99119BFFF718FC13B0F0BD04
:100ED00010B5FFF773FFFFF7B3FF10BD064B10B55A
:100EE0000FCBFFF70BFC054B18780AF01BFCFFF744
:100EF0005FFCFFF7EDFF10BD50130010381300101A
:100F000010B5FFF71FFCFFF79BFF10BD10B50020C9
:100F10000249FFF74DFCFFF793FF10BD0000594059
:100F200000B589B06846FFF703FF009A019B802057
:100F30000399049205930006029A0B1806920793F0
:100F400004980599069A079BFFF7D8FB09B000BDE6
:100F500000B589B06846FFF7EBFE029A039B049246
:100F60000593009A019B0692079304980599069AA7
:100F7000079BFFF7C3FB09B000BD00001FB5064C7F
:100F80006846FFF7D5FE69461022200007F00EFEE6
:100F90000FCCFFF7B3FB1FBD4013001000B589B0A5
:100FA00004A8FFF7C5FE049805990AF055FB40B266
:100FB000FFF7A2FE0022002300900191029203930A
:100FC000009800220199039BFFF798FBFFF738FF79
:100FD00009B000BDF0B504003E4D8DB00A281CD10B
:100FE0003D4B1B78002B18D13C4B1A78002A01D1BD
:100FF00001321A702B78002B0DD1394C2378002B3D
:1010000002D06846FFF794FE00200021FFF7D0FBD6
:10101000012323702B700DB0F0BD2B78002B0ED167
:101020002F4E3378002B02D06846FFF781FE200058
:101030000AF078FBFFF7BCFB01233370EAE7274E89
:101040003578002D21D004A8FFF772FE6B1C68B222
:101050003370FFF751FE06000F0020000AF032FB4C
:1010600032003B0009F0DAF8049A059B08F09AFD7B
:1010700000240023089009910A930B940898099979
:101080000A9A0B9BFFF73AFBC5E708A8FFF750FE4B
:1010900008980999104B00221B78002B18D1114B8E
:1010A00009F0BEFC060020000F000AF00BFB020056
:1010B0000B003000390008F075FD00240023049077
:1010C00005910693079404980599069A079BD9E71A
:1010D000054BE5E7DB05001091060010DA0500106E
:1010E00095060010000024400000304010B5064B6B
:1010F0001B78002B03D00122044B1A7010BD0A206C
:10110000FFF768FFFAE7C046910600108806001056
:1011100010B50920FFF75EFF10BD10B50820FFF7DE
:1011200059FF10BD10B50720FFF754FF10BD000098
:1011300010B5054C0F202378002B00D10938FFF79C
:1011400049FF0023237010BD8806001010B5054C20
:101150000E202378002B00D10938FFF73BFF002336
:10116000237010BD8806001010B5054C0D202378A3
:10117000002B00D10938FFF72DFF0023237010BD8D
:101180008806001010B5054C0C202378002B00D1E8
:101190000938FFF71FFF0023237010BD88060010D9
:1011A00010B5054C0B202378002B00D10938FFF730
:1011B00011FF0023237010BD8806001010B5054CE8
:1011C0000A202378002B00D10938FFF703FF002302
:1011D000237010BD8806001010B50020FFF7FAFE3E
:1011E00010BDF0B589B06846FFF7A2FD00980199DF
:1011F000029C039D04F0F2FC06000F002000290071
:1012000004F0ECFB32003B0009F00AFC049005916D
:101210002000290004F090FC32003B0009F000FCA3
:1012200006900791069A04980599079BFFF766FABE
:1012300009B0F0BD10B5FFF7D4FFFFF783FAFFF751
:10124000BDFDFFF791FDFFF7D1FAFFF741FE10BD9D
:101250001FB5074B1B78002B06D06846FFF768FDCB
:101260000098019905B000BD00200021FAE7C046B2
:10127000DC05001010B5FFF7EBFF0AF0EDF9942341
:10128000421F5B009A4201D2014B187010BDC0464C
:101290002200001010B5FFF7DBFF08F00FF908F08F
:1012A00049F9FFF785FA10BD70B5FFF7D1FF0500CA
:1012B0000C00002200232800210008F067F8002815
:1012C00002D080231B06E41828002100FFF770FAE3
:1012D00070BD000010B5FFF7BBFFE0220B4B1206FC
:1012E00009F00AFEFFF764FA094B0A4A18605960D0
:1012F00000210020084B1860596000230121137061
:10130000064A1170064A137010BDC0464D62603F18
:10131000301300101F11001080060010A6060010E8
:101320008C06001010B520220021134807F05FFC46
:10133000FFF78EFF114C20606160FFF789FFFFF718
:1013400037FA02000B000E490A604B6020686168A2
:1013500009F0D2FD00220B4B08F060FF01220A4B7E
:1013600018605960094B1A700023094A1370094A22
:101370001370094A137010BDD4060010C80600107F
:10138000C006001000003F40780600109C060010C8
:101390008C060010AD0600101F11001010B5FFF7ED
:1013A00057FF8022034B120608F038FFFFF700FAC0
:1013B00010BDC0465347E13F10B5FFF749FFE0229B
:1013C000034B120608F02AFFFFF7F2F910BDC046E2
:1013D00045E2E33F10B5FFF73BFF8022034B1206C7
:1013E00009F01EFBFFF7E4F910BDC046EB510440C5
:1013F00010B5FFF72DFF0022024B09F011FBFFF79C
:10140000D7F910BD86480E4010B5FFF721FF002226
:10141000054B09F071FDC022044B120608F0FEFED8
:10142000FFF7C6F910BDC04600004040CCCCFC3FE1
:1014300010B5FFF70DFF8022034B920508F0EEFE7A
:10144000FFF7B6F910BDC04611A3014010B5FFF774
:10145000FFFE0022054B09F0E3FAC022044BD2053F
:1014600008F0DCFEFFF7A4F910BDC046008066401E
:10147000FB210940F7B5FFF7EBFE1D4A1D4B08F0B5
:1014800091FB0D0004000AF0E7F80AF01BF9009048
:10149000019102000B002000290009F02DFD00221F
:1014A000154B09F0BDFA0D0004000AF0D5F80AF05A
:1014B00009F906000F0002000B002000290009F0C6
:1014C0001BFD00220C4B09F0ABFA00220B4B08F07D
:1014D000A5FE32003B0008F065FB0022074B08F038
:1014E0009DFE009A019B08F05DFBFFF761F9F7BDD7
:1014F000BBBDD7D9DF7CDB3D0000594000004E402A
:10150000F8B5FFF7A5FE06000F00FFF7A1FE07F0F4
:10151000D5FF05000C003000390007F0CFFF284050
:101520002140C043C94308F005F8FFF741F9F8BD71
:10153000F8B5FFF78DFE07F0A3FFC4B2FFF788FEF2
:1015400007F09EFFC5B200202C1B0B49E4B201340A
:10155000FFF72EF9631EDBB29D4200D8F8BDFFF7FE
:1015600077FE06000F0020000AF0ACF832003B00C6
:1015700009F056FAEBE7C0460000F03FF8B5FFF778
:1015800067FEFFF715F907F07BFF0124C5B2FFF7EF
:10159000CFFFAC4200D9F8BDFFF75AFE060020008D
:1015A0000F000AF08FF802000B003000390008F03D
:1015B00035FE0134FFF7FCF8E4B2EAE710B5FFF7B7
:1015C00047FE8022034B120609F02AFAFFF7F0F8D3
:1015D00010BDC0465347E13F10B5FFF739FEE0228A
:1015E000034B120609F01CFAFFF7E2F810BDC046E3
:1015F00045E2E33F10B5FFF72BFE8022034B1206B6
:1016000008F00CFEFFF7D4F810BDC046EB510440C3
:1016100010B5FFF71DFE0022024B08F0FFFDFFF79B
:10162000C7F810BD86480E4010B5FFF711FEC02266
:10163000054B120609F0F4F90022044B08F0B2FA47
:10164000FFF7B6F810BDC046CCCCFC3F00004040D0
:1016500010B5FFF7FDFD8022034B920509F0E0F97C
:10166000FFF7A6F810BDC04611A3014010B5FFF763
:10167000EFFDC022054BD20509F0D2F90022044B40
:1016800008F0CCFDFFF794F810BDC046FB210940DF
:1016900000806640F0B585B0FFF7DAFD0022284BE8
:1016A00009F0BEF9274A284B08F07CFA0022244BA7
:1016B00004000D0008F0B2FD09F0CEFF0AF002F8B8
:1016C00000221F4B0090019109F0AAF902900391AA
:1016D00002000B002000290009F00EFC00221B4B29
:1016E00008F09CFD09F0B8FF09F0ECFF0022174B51
:1016F00006000F0009F094F902000B0020002900F9
:1017000009F0FAFB029A039B09F0F6FB0022104B4A
:1017100008F084FD002204000D00300039000D4B5C
:1017200008F07CFD009A019B08F03CFA02000B00D7
:101730002000290008F036FAFFF73AF805B0F0BDAE
:101740000020AC40BBBDD7D9DF7CDB3D00004E4064
:101750000088C3400000594030B5264A264B127815
:101760001B7885B0002A19D0002B0ED0FFF770FD32
:101770000022224B09F054F907F0A0FE0B000343AE
:1017800035D1FEF76DFD05B030BD6846FFF7D0FAE4
:10179000102269461A4807F009FAF4E7002BF4D042
:1017A000184A107800281BD0431EDBB21370002BA0
:1017B000E9D0023840B2FFF79FFA04000D00FFF7AE
:1017C00047FD22002B0009F02BF907F077FE07F008
:1017D000B1FE22002B0008F021FDFEF7E9FFD2E761
:1017E000FFF736FD0022084B08F018FDC4E707F0AC
:1017F000A1FEF2E791060010DB0500100000B03FEB
:10180000B0060010DA0500100000244010B5FFF704
:101810001FFD07F035FEC0B2072803D8024B187031
:1018200006F00AF910BDC0469D01001010B5FFF783
:101830000FFD07F025FEC0B23F2803D8024B1870F9
:1018400006F0FAF810BDC046C81A001010B5040022
:1018500074280CD9212C17D0FEF702FD193CE4B2F4
:101860000B2C11D80D4BE340DB0716D40CE00C4BCE
:101870001A78272353430B4A1B189B009B58984701
:101880000A2CEBD9122CE5D10023074A1370044A25
:101890001370064A1370064A137010BD210C000025
:1018A0008C060010A0BC00009D06001093060010DE
:1018B00092060010F0B52E4AC30085B0D3181A68FE
:1018C0005B68040000920193FEF7CEFD0500FEF771
:1018D000C7FCFEF77BFD274B6E1C5F5DFF2F10D111
:1018E000FFF7B6FC224BE4001C1920606160009AEF
:1018F000019B09F001FB02000B0009F091F805B013
:10190000F0BDFD2F1DD11C4F9E5D3B780235042B91
:1019100007D91A480422411C07F08BF93B78013B98
:101920003B70154A1378591C1170144AD654104B49
:10193000F6009E1930687168FEF73AFF2E003500F8
:10194000C9E70F4B06221D7827230E4902A85D43E5
:1019500007F02CF900237D19EDB202AAD25CAA424D
:10196000EDD00133062BF8D13800FFF76FFFE6E723
:10197000201100105F080010590800105A080010CC
:101980008C06001083BA0000F8B52025002400263C
:1019900000272000FEF790FD00280AD12000FFF765
:1019A00089FF02000B003000390008F0FBF8060048
:1019B0000F000134E4B2202CEBD1E02230003900DA
:1019C000054B120607F0E2FC002803D1013DEDB201
:1019D000002DDBD1F8BDC0464D62503F70B50D4EB5
:1019E00034782000FEF740FD0B4B1B5CFF2B02D030
:1019F0002000FFF755F80024084D013DE2B2013404
:101A0000295DFF2902D1FFF7BFFF70BD3078FEF7D7
:101A100019FFF3E7281300105F08001034080010C6
:101A2000F7B5012006F0D6F804002220002C1DD1C5
:101A30002500174B0193019B01221E785F7830002F
:101A4000390006F023FC39003000002206F06AFC61
:101A5000271D104EFFB2F179B07906F039FC00284D
:101A600005D12800FEF7DAFD0B4B185DFEBD0134F1
:101A7000E4B2023EA742EED12800FEF7CFFD019B63
:101A800001350233EDB201930A2DD4D1FF20EDE7E9
:101A9000B4C20000ACC2000084C2000070B50024D3
:101AA000FFF7BEFF0500012006F010FEFF2D00D05D
:101AB00000240134E4B2032CF2D170BD00B50C4B0C
:101AC00089B01B78012B11D96846FFF731F904A8BA
:101AD000FFF72EF900980199029A039BFEF70EFE7C
:101AE00004980599069A079BFEF708FE09B000BD09
:101AF000DC05001010B5FFF7E1FFFFF7A9FB124C62
:101B000020606160FFF7A4FBFEF752FE2268636865
:101B100009F0F2F900220D4B08F082FF00220C4B75
:101B200008F07CFB0B4B012218605960002000215B
:101B3000094B18605960094B1A700023084A13704A
:101B4000084A137010BDC046C00600100000E03FF8
:101B50000000244078060010800600109406001053
:101B60008C0600101F11001000B58BB0FEF74AFB69
:101B7000002815D006A8FFF7DBF880200799069A01
:101B800000060B180292039300220023049205938F
:101B9000002202980399059BFEF7B0FD0BB000BD33
:101BA00002A8FFF7C5F8802000068446039B029A2E
:101BB0000193019961440B00059906920793049AD9
:101BC0000B180892099306980799089A099BE3E76E
:101BD00010B5FFF7C9FFFFF7C7F810BD10B5FEF746
:101BE000B1FDFFF757FBFFF7F3FF10BD10B5002065
:101BF0000249FEF7DDFDFFF7EBFF10BD0000F03FEF
:101C0000274B70B50FCBFEF779FD264E307809F0E3
:101C100089FDFEF7CDFDFFF713F9234C20686168BD
:101C2000A268E368FEF76AFD204D28686968AA6823
:101C3000EB68FEF763FDFFF703F9FFF7C9FF1C4BE5
:101C40000FCBFEF75BFD307809F06CFDFEF7B0FDC1
:101C5000FFF7F6F820686168A268E368FEF74EFDBA
:101C6000FEF770FDFFF7ECF8FFF7B2FFFFF730F972
:101C7000FEF768FD0FCCFEF741FDFFF7E1F8FFF737
:101C800073FF0FCDFEF73AFDFFF76EF8307809F0DD
:101C900049FDFEF78DFDFFF71BF9FFF70FFF70BD44
:101CA0007013001038130010501300108013001030
:101CB0006013001010B5FFF794FAFEF743FDFFF72D
:101CC0007DF8FFF751FFFFF74FF8FEF78FFDFFF7A5
:101CD000FFF810BD00B5114B8DB01B78022B1AD93F
:101CE0006846FFF725F804A8FFF722F808A8FFF7D1
:101CF0001FF800980199029A039BFEF7FFFC0898D1
:101D000009990A9A0B9BFEF7F9FC04980599069A23
:101D1000079BFEF7F3FC0DB000BDC046DC050010CC
:101D200010B5FFF7D7FFFFF7D5FF10BD10B5FFF7D0
:101D3000C5FEFEF707FDFFF7F3FFFFF7BFFEFFF756
:101D400047FFFFF7BBFEFFF7C3F8FFF7DFF810BD53
:101D50007FB51025324E3378013B3370FEF7F2FC2D
:101D6000304CE3686168A2682068FEF7C7FCFFF7A3
:101D7000A5FEFFF72DFF6846FEF7DAFF2A00694649
:101D8000200006F013FFFEF7DDFCFEF7DBFCFFF79B
:101D900057F8254CE3686168A2682068FEF7AEFC3E
:101DA000FFF78CFEFFF714FF6846FEF7C1FF2A001D
:101DB0006946200006F0FAFEFFF780FEFEF7C2FC3F
:101DC000FFF7AEFFFFF73CF8184CE3686168A268C4
:101DD0002068FEF793FCFFF771FEFFF7F9FE6846F7
:101DE000FEF7A6FF2A006946200006F0DFFE104C31
:101DF000E3686168A2682068FEF780FCFFF75EFE7A
:101E0000FFF7E6FE6846FEF793FF2A0069462000CA
:101E100006F0CCFE307809F085FCFEF7C9FC7FBDEA
:101E200038130010501300106013001070130010CE
:101E3000801300107FB510252E4E33780133337098
:101E4000FEF780FC2C4CE3686168A2682068FEF70E
:101E500055FCFEF789FF6846FEF76AFF2A006946CF
:101E6000200006F0A3FEFEF76DFCFEF76BFCFEF70C
:101E7000E7FF224CE3686168A2682068FEF73EFC39
:101E8000FEF772FF6846FEF753FF2A0069462000FE
:101E900006F08CFEFFF712FEFEF754FCFFF740FF42
:101EA000FEF7CEFF164CE3686168A2682068FEF773
:101EB00025FCFEF759FF6846FEF73AFF2A006946FF
:101EC000200006F073FE0F4CE3686168A26820688A
:101ED000FEF714FCFEF748FF6846FEF729FF2A00CC
:101EE0006946200006F062FE307809F01BFCFEF720
:101EF0005FFC7FBD381300105013001060130010FA
:101F0000701300108013001070B5124B1B78002B5B
:101F100012D0FEF707FB05000C00FEF703FB0200E2
:101F20000B002800210007F07DFA6422002307F04F
:101F300055FAFEF7BDFC70BDFEF7F4FA05000C0083
:101F4000FEF7F0FA02000B002800210007F06AFA01
:101F5000EFE7C0462100001010B51A4B1B78002B8C
:101F600016D0FEF7DFFA43B2020601D5404243B273
:101F700001200021013B5BB25A1C04D1FEF798FC02
:101F8000FFF7C2FF10BD020F090111430001F1E785
:101F90000D4B1B78002B0FD0FEF7C4FA64220023F0
:101FA00007F01CFA40B2FEF7A7FE0022074B08F02C
:101FB00037FD07F083FAE1E7FEF7B4FA40B2FEF727
:101FC0009BFEF6E79106001021000010000059402A
:101FD00070B50D4B1B78002B03D00C4B01221A70EF
:101FE00070BD0B4C2378002B0CD10A4D2B78002BA5
:101FF00001D0FEF797FA00200021FEF759FC0123DB
:102000002B702370044BE9E791060010880600103E
:102010009219001091190010AA060010F7B5364A5F
:10202000364E127833780190002A26D0002B3FD00C
:10203000FEF778FA6422002305000C0007F0CEF9C1
:102040000A22002307F0EEF906000F002800210005
:102050000A22002307F0C2F9002530003900D4B26B
:1020600000230A220019694107F0DCF92B00019ACC
:1020700080185941FEF71CFC1AE021491500097827
:10208000019C0091002B17D11E4F3B78002B01D0F3
:10209000FEF748FA009B002B0BD06422002320009F
:1020A000290007F0BFF9FEF703FC01233B703370F2
:1020B000F7BD20002900F6E7009B002B0CD0FEF7AF
:1020C00031FA0A22002307F089F9642200196941D4
:1020D000002307F0A7F9CDE7FEF724FA0A4B1022F8
:1020E0001E780023002E01D10A22002307F09AF95E
:1020F00000196941BEE7C046AA06001092190010F7
:1021000021000010911900109106001010B509204F
:10211000FFF784FF10BD10B50820FFF77FFF10BD4B
:1021200010B50720FFF77AFF10BD000010B5054C71
:102130000F202378002B00D10938FFF76FFF002311
:10214000237010BD8806001010B5054C0E202378B2
:10215000002B00D10938FFF761FF0023237010BD69
:102160008806001010B5054C0D202378002B00D1F7
:102170000938FFF753FF0023237010BD88060010B5
:1021800010B5054C0C202378002B00D10938FFF73F
:1021900045FF0023237010BD8806001010B5054CC4
:1021A0000B202378002B00D10938FFF737FF0023DD
:1021B000237010BD8806001010B5054C0A20237846
:1021C000002B00D10938FFF729FF0023237010BD31
:1021D0008806001010B50020FFF720FF10BDF7B5EE
:1021E000FEF7A0F907000E00FEF79CF900900191A0
:1021F000FEF798F905000C0038003100FEF758FB97
:1022000028002100FEF754FB00980199FEF750FBCF
:10221000F7BDF8B5FEF786F907000E00FEF782F964
:1022200005000C0038003100FEF742FB28002100B9
:10223000FEF73EFBF8BD0000F0B58DB0FDF7E2FF04
:10224000002810D0FFF704F8C0222C4BD20508F06C
:10225000E7FB00222A4B07F0E1FF03F06DFCFEF7DD
:10226000A7FA0DB0F0BD04A8FEF762FD0698079925
:10227000049C059D03F0B2FC06000F00200029001D
:1022800003F05AFC3200029003913B0000201D49EC
:1022900007F0C4FF0090019102000B0030003900EC
:1022A00007F080FC029A039B08F0BAFB0022164B51
:1022B00008F0B6FB08900991C02022002B001349BA
:1022C000C00508F019FE03F037FC009A019B0400DA
:1022D0000D003000390008F00FFE22002B0008F03E
:1022E0009FFB0022084B08F09BFB0A900B910A9A77
:1022F000089809990B9BFEF701FAB2E7FB21094008
:10230000008066400000F03F0000E03FFB21F93F05
:10231000F0B58DB0FDF776FF002810D0FEF798FFDE
:10232000C0222E4BD20508F07BFB00222C4B07F07D
:1023300075FF03F053FBFEF73BFA0DB0F0BD04A8A8
:10234000FEF7F6FC06980799049E059F03F046FCED
:102350000400C0200D0032003B002249C00508F0F7
:10236000CBFD03F0E9FB2200029003912B0000203B
:102370001D4907F053FF0090019102000B0020005F
:10238000290007F00FFC029A039B08F049FB00228A
:10239000164B08F045FB089009913000390003F016
:1023A000CBFB80231B06CE180700009A019B200060
:1023B000290008F0A1FD02000B003800310008F0F0
:1023C0002FFB0022094B08F02BFB0A900B910A9A75
:1023D000089809990B9BFEF791F9AEE7FB2109409C
:1023E00000806640FB21F93F0000F03F0000E03F25
:1023F00070B5064C0500200006F031FC691C421B3C
:102400006118601906F0D2FB70BDC046630600106B
:1024100070B50D0004000A21280006F0B1FE30312D
:1024200020236170092D0AD90A21280006F022FE16
:102430000A21C0B206F0A4FE0B003033DBB22370D9
:1024400070BD000010B5FFF739FBFEF77BF9FFF711
:1024500067FC00200349FEF7ABF9FEF739FDFEF7F4
:10246000EFFC10BD00005940F0B52C4B85B00700C3
:1024700018780291FDF7F8FF00231C001D0003905F
:102480000193039BE918264B5A5CFF2A02D101985D
:1024900005B0F0BDFD2A22D1212CF2D85B18032112
:1024A0005B783A1919409B08313353704131029BD4
:1024B0001170A21CD2B2002B0DD01A4B1B78002B2E
:1024C00009D0023B9D4206D103347F213800E4B29B
:1024D000FEF704F9220002351400EDB2D1E7222CF8
:1024E000CFD8114B661C9B5CF6B23B55029B002B70
:1024F0000FD00C4B1B78002B0BD0013B9D4208D119
:10250000023432007F213800E4B2FEF7E7F801968A
:10251000260001353400EDB2B3E7C04628130010A1
:102520005F08001060060010C8C2000070B50024EB
:102530008AB003AD18222021280006F058FB20495C
:1025400001AE0622300008312C7606F02FFB1D4B21
:102550001A78A24210D0335D1B49A2009B002800CC
:10256000D2B2C9180134FEF74FFA062CF3D1280075
:10257000FEF756FA0AB070BD144B1C78002C0DD033
:102580001400335D1249A2009B002800D2B2C91882
:102590000134FEF739FA062CF3D1E8E70D4A127838
:1025A000002AE4D0335D0C49A2009B002800D2B27F
:1025B000C9180134FEF728FA062CF3D1D7E7C04634
:1025C00080BC00009A060010230000109F06001037
:1025D0006D000010A806001085010010F0B54A4EED
:1025E0008DB03378002B41D0FDF70CFE00283DD094
:1025F000FEF72EFE337804000D00002B30D0FDF7DF
:1026000001FE00282CD0FEF723FE404B1B78002B48
:102610000AD0089409950A900B91089809990A9A8A
:102620000B9BFEF76BF81FE0C022394BD20508F078
:10263000F7F90022374B07F0F1FD06000F0003F019
:10264000CDF922002B0008F0EBF908900991300039
:10265000390003F071FA22002B0008F0E1F9DAE703
:1026600020002900FEF7A4F80DB0F0BD6846FEF783
:102670005FFB009C019D029E039F244B1B78002B57
:1026800014D0002200230496059716001F0006921E
:102690000793069A079B04980599FEF72FF83200D6
:1026A0003B00089409950A920B93B6E732003B0071
:1026B00020002900FEF784FA0022002304900591EF
:1026C0000692079304980599069A079BFEF716F859
:1026D00022002B002000290008F0A2F9320004009B
:1026E0000D003B003000390008F09AF902000B00A1
:1026F0002000290007F056FA03F0DEFA002200233A
:1027000008900991CFE7C046DC05001020000010BA
:10271000FB21094000806640F0B58BB002A8FEF7AF
:1027200007FB029E039F049C059D32003B00300086
:10273000390008F075F92200009001912B0020006B
:10274000290008F06DF902000B000098019907F0CC
:1027500029FA03F0B1FA03F079FA22000690079102
:102760002B0030003900FEF72BFAC022084BD205AF
:1027700008F056F90022074B07F050FD0890099128
:10278000089A06980799099BFDF7B8FF0BB0F0BDB2
:10279000FB2109400080664010B5FFF7BDFF002017
:1027A0000349FEF705F8FFF7B7FFFEF791FB10BDF1
:1027B0000000244010B5FEF7F7FAFDF7C3FFFDF760
:1027C000C1FFFDF7BFFFFDF7BDFF00201849FDF772
:1027D000EFFFFEF735FBFFF771F900201549FDF714
:1027E000E7FFFEF72DFBFEF7E9FAFFF7F1F9FEF739
:1027F000E5FAFEF7B9FAFFF78FFFFFF7F7F9FEF7F3
:102800001FFBFFF75BF9FFF787FFFFF7ADF9C0206C
:102810000949C005FDF7CCFFFFF77EFFFEF7A4FADC
:10282000FDF7E4FFFEF754FBFEF79EFA10BDC0462D
:102830000000284000002440FB21194030B58DB035
:102840006846FEF775FA04A8FEF772FA049805992F
:102850000022002306F094FD0024002500282AD041
:102860000698079922002B0006F08AFD002822D046
:102870000098019922002B0006F082FD002815D057
:102880000298039922002B0006F07AFD00280DD053
:102890001022124908A8891806F088F908980999A1
:1028A0000A9A0B9BFDF72AFF0DB030BD08940995DD
:1028B0000A940B95F2E704980599069A079BFDF791
:1028C0001DFFFFF729FF00980199029A039BFDF76E
:1028D00015FFFEF7B5FAFEF784FCE5E780BC0000C3
:1028E00010B5FFF7EBF800200D49FDF761FFFEF78B
:1028F000EFFAFDF727FFFFF7EDF9FEF755FAFFF7BF
:10290000DDF8FFF79BFFFDF71DFFFFF76FF9FFF7FE
:10291000D5F8FEF7DDFAFFF7D1F8FEF7D9FA10BDCA
:102920000000594010B500200449FDF741FFFFF7B2
:10293000F3FEFEF785FAFEF754FC10BD00002440BC
:102940001FB56846FEF7F4F90098019900220023AC
:1029500006F016FD002805D000200021FDF728FF15
:1029600005B000BD029A039B00980199FDF7C6FED1
:10297000FFF7D2FE00200449FDF71AFFFEF760FAC8
:10298000FEF72FFCECE7C0460000E03F10B5FFF774
:1029900095F8FDF72BFFFEF79BFAFDF7D3FEFDF749
:1029A000D1FEFEF74DFAFFF7BBF9FFF711F9FFF77C
:1029B000C7FFFDF7C7FEFFF7B3F9FFF7D5F8FDF73F
:1029C000C1FEFFF7ADF9FEF7CFF9FFF783F9FFF787
:1029D00075F8FFF7FDF810BD10B5FEF77FFAFDF7AB
:1029E000B1FEFEF72DFA0E4C207808F09BFEFDF7A5
:1029F000DFFEFEF725FAFFF7B7F80A4B0FCBFDF71E
:102A00007DFEFEF7B1F9207808F08CFEFDF7D0FED0
:102A1000FFF7ECF8FEF75CFAFFF792FF10BDC04637
:102A2000381300106013001010B5FDF78BFEFEF791
:102A300067FAFFF799F8FEF7B7F9FFF781FFFFF79D
:102A40003DF8FDF7DBFEFEF7FBF9FEF78DF9FFF72A
:102A500063FEFDF7D3FEFFF787F8FEF7F1F9FDF708
:102A6000D1FB00280CD0FEF7F3FB0022054B07F04A
:102A7000D7FFC022044BD20507F0D0FBFDF798FE2C
:102A800010BDC04600806640FB21094010B5FFF72D
:102A9000CBFFFFF769F8FDF7B5FB002806D0002053
:102AA0000449FDF785FEFEF75FF910BDC02002491D
:102AB000C005F6E700805640FB21F93F10B5FDF751
:102AC00041FEFEF71DFAFEF76FF9FFF739FFFEF73B
:102AD00075F9FEF7B5F9FFF7A7FF10BD10B5164B56
:102AE0001B78002B0AD0FDF72DFEFFF7E3F8FEF769
:102AF000E5FFFEF79FFBFEF7EBF913E00F4B1B78AA
:102B0000002B10D0FDF71EFEFEF74EF9FEF7D6FFA4
:102B1000FFF72AF8FEF748F9FEF7DAF9FFF710FF9A
:102B2000FFF7FAFD10BDFDF70DFEFFF785FBFEF781
:102B3000C5FFFFF7EDFBDEE79206001093060010DD
:102B400010B50D4B1B78002B02D0FEF773FB10BDA8
:102B50000A4B1B78002B0CD0FDF7F4FDFEF7D0F9E3
:102B6000FFF744F8FFF7ECFEFEF7FEF8FFF7D4FDA1
:102B7000EDE7FFF7CDFBEAE79206001093060010A1
:102B800010B50D4B1B78002B02D0FFF793F810BD4A
:102B90000A4B1B78002B0CD0FDF7D4FDFEF7B0F9E3
:102BA000FEF702F9FFF7CCFEFEF7DEF8FFF7B4FD03
:102BB000EDE7FFF741FBEAE79206001093060010ED
:102BC000F0B58FB00BAC0190029105922021082244
:102BD0002000089306F00BF800232372734B0022A9
:102BE0001B780493002B3CD000230198029906F037
:102BF000CDFB8022029B12069D18002800D11D00EB
:102C0000290000226A4B019806F0C0FB0BAD00289A
:102C100008D030232B702000089A0599FDF7C6FADA
:102C20000FB0F0BD0198029906F066FC0F27030073
:102C30000DA81A000A4300D1FAE2A84203D15D4967
:102C400006F015F8E7E71E003E4032003032392A20
:102C500000D92732013802701B090A0713430909FA
:102C6000E7E700230198029906F090FB019D0028F8
:102C700059D080220A27029B12069C1821004E4A36
:102C80004E4B019806F0A0FB00282BD121004C4AA6
:102C90004C4B019806F084FB002807D0002200234B
:102CA0002100019806F086FB00281BD1019A230021
:102CB0001000210008F0B2FC002813D101226600A8
:102CC00076083100404B0198524208F0A7FC0028DA
:102CD0002CD1012231003C4B0198524206F060FB9E
:102CE000002823D133490BA805F0C1FF0BA8FDF73D
:102CF00073FE06260BAD2878002800D190E7334BF1
:102D000005991C782E2804D1091BC9B20A1BD3B21D
:102D100005937443089AFDF7D3F9059B01351C19F7
:102D2000E3B20593E7E70127029CA7E72100244AC5
:102D3000244B019806F02AFB00281AD12100244ACE
:102D4000244B019806F040FB002800D184E13800B4
:102D500008F0B8FC02000B0000201F4907F05EFAE3
:102D600002000B000198210006F010FB002800D1A2
:102D700072E1002200232100019806F001FB0028E7
:102D800000D108E130230BAA1370144B19780029E5
:102D900001D02E2313700123302001E0D0540133E1
:102DA000DCB2A142A2D9082BF8D19FE7910600100E
:102DB0000000F03F8ABA00007DC39425AD49B254AB
:102DC0003EC3D84E7D7F612BFFFFEF7F1B000010BD
:102DD000FCA9F1D24D62503FD0126341DA050010D8
:102DE00028002100964B002207F01AFE0C00050077
:102DF0000398013843B20393002228002100914B2D
:102E000006F0C4FA0028EBD16B461B7B0022079327
:102E1000280021008B4B06F0D7FA002209900028E9
:102E200000D0BAE000230299019806F0AFFA431EE1
:102E300098410723181AC3B20693FDF75DFF0200FD
:102E40000B002800210007F0EBFD00227E4B06005E
:102E50000F0006F0A7FE08F0FFFB39000400300069
:102E600008F0FAFB0A2705002000099E002800D080
:102E70009FE00A27002D00D0A1E0049BB34208D2B6
:102E800020000A2106F080F904000798013043B2BF
:102E900003936B461D7B069B581B40B2FDF72CFF2E
:102EA00006000F00200008F00DFC3B00320007F088
:102EB000B5F908F0D1FB39000490300008F0CCFBE4
:102EC0000100200006F046FA039B0C00002B13DAE9
:102ED000684240B2FDF710FF06000F00200008F026
:102EE000F1FB32003B0007F099F90022564B06F047
:102EF00059FE08F0B1FB04006B46039A1B7B002AC5
:102F000000DA0023069AD31ADBB203934F4B1B78E7
:102F10000693002B00D181E04D4B1D78002D7ED013
:102F20000BAF3D000A264B4B039A1B78D31A07932D
:102F30007B1B0399DAB291424BD80B000DACE41A1B
:102F40002E230A25013C2370049B002B6AD100220A
:102F500000230198029906F019FA002802D02D23C7
:102F6000013C2370069B002B04D0394B1B78002BAF
:102F700000D0BBE6200005F072FE00220138C0B28E
:102F80002018844200D1B1E60378302B00D0ADE6A2
:102F900002700138F5E703902EE728002100284B46
:102FA00007F03CF9050007980C00013043B2039389
:102FB0002AE73900013606F0E7F8F6B256E72800AE
:102FC000390006F0E1F8049B05000133DBB20493FD
:102FD00050E7079A20219A4205DA3100200006F0D6
:102FE000B9F93031C9B2E9712000310006F0CCF8EE
:102FF000013D04009CE72000390006F0ABF93031B8
:1030000020003170390006F0BFF804000135EDB240
:10301000039B013EAB42EED10DAC90E7069D0A2723
:103020000DAEF5E70498290006F094F9013C303123
:1030300004982170290006F0A7F8049084E7C046A0
:10304000000024400000F03F0000E03FDB050010DE
:103050009E060010DA050010002300220198029954
:1030600006F094F9431E984100270600002228002C
:103070002100714B06F08AF9002800D0A7E0002259
:10308000280021006C4B06F09FF9002800D0A8E032
:103090003B0008330730122B00D80820861BF3B200
:1030A0000393039BD81E40B2FDF726FE02000B00DF
:1030B0002800210007F0B4FC0022604B04000D0042
:1030C00006F070FD08F0C8FA29000600200008F09C
:1030D000C3FA002504003000002800D08BE0002C4B
:1030E00000D08EE0049BAB4205D230000A2106F0EE
:1030F0004BF806000137039B181F40B2FDF7FCFD9B
:103100000D000400300008F0DDFA2B00220007F06B
:1031100085F808F0A1FA29000490200008F09CFA34
:103120000100300006F016F9FB0F0D0006937C1E1F
:1031300001D50124E41B0A21200006F00BF90BAF96
:103140003031F97120000A2106F01EF80B260AAB77
:10315000F618002807D00A2106F0FCF80A263031BC
:103160000AABB971F618069A2B23013E002A00D04B
:10317000023334000A273370039B043B0693280074
:103180003900039406F0E6F8013C30312800217044
:10319000390005F0F9FF331B069ADBB205009342B4
:1031A000EDDB2E23013C23700A24039D023D049B8A
:1031B000002B30D1002200230198029906F0E6F896
:1031C000002800D192E52D23013D2B708EE52800CB
:1031D000210000221A4B07F023FC013F05000C00E0
:1031E00044E7280021000022154B07F017F80137AB
:1031F00005000C0043E70A21013505F0C5FFEDB2DB
:103200006AE720000A2105F0BFFF049B0400013398
:10321000DBB2049363E70498210006F09BF8013DBC
:10322000303104982970210005F0AEFF0490BEE70C
:103230002800FDF7D1FBEEE40000F03F0000E03F86
:1032400000002440F7B50C0015000090FDF734F99C
:10325000002822D00098FDF707F9230027001C4E14
:103260002A33DBB2361801937078FF2809D0390071
:103270002A00FCF725FF0637019BFFB201369F426B
:10328000F2D1144B009A1B78934205D1063C2A00D8
:10329000B220E1B2FCF714FFF7BD009BDA000E4B41
:1032A0009B181E685F68002200233000390006F07A
:1032B00067F8002805D02A002100CC20FCF700FF89
:1032C000DFE72B00220030003900FFF779FCD8E758
:1032D0005F080010281300102011001070B5174B64
:1032E0001C78174B1B78002B03D0032C01D9043C0E
:1032F000E4B2144B1B78002B03D0002C01D0013C0E
:10330000E4B20025104E2A00200006213570FFF798
:1033100099FF601C2A003B21C0B2FFF793FF0135E3
:10332000201D2A000621C0B205343570FFF78AFF40
:103330002A003B21E0B2FFF785FF70BD2813001083
:103340002A130010291300106106001010B50A4B53
:103350001B78002B03D00948FDF762FB10BD084B1A
:10336000084A1B781278134302D0FFF7DFF8F5E71D
:10337000FFF7B4FFF2E7C046A30600108EBA0000C4
:10338000A506001097060010F7B5FDF761FF0D00C8
:10339000040004F071FD684601A904F015FE29003F
:1033A000200006F06DF880266B461A4FC0B21880D8
:1033B000F60529002000FDF7FBF9FEF70FFC3000B1
:1033C0003900FDF7F5F9FDF7CFFCFDF79FFDFDF79F
:1033D0003FFF06F055F86B46290098702000FDF776
:1033E000E7F9FDF793FDFEF7F9FB30003900FDF733
:1033F000DFF9FDF7B9FCFDF789FDFDF729FF06F0C0
:103400003FF86B460022D87001A9684604F020FE00
:10341000F7BDC046E17A743F37B5FDF719FF0D00DF
:10342000040004F029FD684601A904F0CDFD29003F
:10343000200006F025F86B4680222900D20518717D
:103440000B4B200006F0AEFBFDF7B2F9FEF7C6FB12
:10345000FDF7FEFE0022074B07F0E2FA06F010F837
:103460006B460022587101A9684604F0F1FD37BD92
:10347000E17A743F0000594013B504F0FDFC01A946
:10348000684604F0A1FD6B46987806F03DFB1649AE
:1034900006F022FA6B46041C188806F035FB011C66
:1034A000201C06F07BF86B46041CD87806F02CFB39
:1034B0000E4906F011FA011C201C06F06FF8041CDE
:1034C000684604F0F5FD072105F044FF080006F00A
:1034D0001BFB074906F000FA211C06F05FF808F014
:1034E00047F9FDF765F913BD0000C84200401C46CE
:1034F0000050C34707B504F0BFFC684601A904F0BB
:1035000063FD6B463C205B7958436B469B79C01842
:103510000EBD10B5FEF7C2FA04F048FD04F061FAE2
:103520000020012105F0A0F8002004F053FB002842
:1035300002D1012105F098F804F0A4FA10BD0000B2
:10354000F8B572B6B120FDF79BF80020FDF798F8AA
:103550001020FDF795F8E020FDF792F80024144DB7
:1035600001222E5D0021022004F0DCFE0134300037
:10357000FDF768F8842CF2D1B020FDF781F8002027
:10358000FDF77EF81020FDF77BF88426E020FDF79C
:1035900077F876002F5D01220021022004F0C2FEA0
:1035A00001343800FDF74EF8B442F3D162B6F8BDED
:1035B00020120010F0B59FB005F076FB04F0CAFAB7
:1035C0000021DC4804F0D0FE0021DB4804F0CCFEF2
:1035D00004F02BFB01220421002004F057FE0022FE
:1035E0000421100004F09EFE01220521002004F0B9
:1035F0004DFE00220521100004F094FE002004F08E
:1036000089FDA022FF215200CC4805F0F0FAF022FB
:10361000FF21D200CA4805F0EAFAFFF76BFF00234A
:1036200007900393C74B1B68002B50D0C64B1C78E8
:10363000002C47D184222100C448520005F0D7FA5B
:10364000C34BC44D1E782C70002E00D1A9E0C24D92
:10365000C24B28001C7005F002FB002800D19AE044
:10366000BF4E7F2128003278FDF738F8280022006D
:103670000321FCF79BFD3078FEF7BAFE01220325FB
:10368000B64B1A70B74B0122187829000001203080
:103690002018C0B2FCF714FDB34B1B78A34206D12F
:1036A0000635EDB2012229007F20FCF709FD013427
:1036B0000635E4B2EDB2102CE4D1AC4B1B78002BF4
:1036C00000D1E6E1FFF73CFF00229E4B1A60A849BB
:1036D000A84F0B780093002B01D100F007FEA64AFB
:1036E000A6481378C05C3870FF2803D0312B01D86E
:1036F00000F0F6FD00230B70FEF7D0F9A04BA14AB5
:103700001B7812781343A04A127813439F4A127809
:103710001343FF220392002B02D18A4BFE3A1A6018
:10372000FFF7E8FE079B934FC01A994B1B7898420E
:1037300001D922233B703878FF2829D0039B984277
:1037400026D08B4B8E4A1B78127813438D4A127801
:1037500013438D4A127813438C4A1278134302D1D3
:103760000122784B1A608B4B1B78002B05D0824AC4
:103770001378591C1170814AD054222801D000F0CE
:10378000F1FFFF233B70FFF7C4FEFFF7B3FE079086
:10379000784B1B7845E7220003217F20FCF790FC43
:1037A0006CE77D4B1F78002F28D001257B4C7C4B8C
:1037B00022786A4FD2009B18186859680322330098
:1037C0003E70FFF7FDF92A000321B3203D70FCF79E
:1037D00077FC247814AF61193800C9B2BE70FEF7C7
:1037E00017FE2A000F213800FCF7E0FC2A002121F7
:1037F0006C4BA400E058FCF7D9FC5EE75B4B1B78F0
:10380000002B71D0684E694B1C685D683268736824
:103810002000290007F070FB02000B0020002900A7
:1038200006F0FCFC0022624B07F0FAF805F028FED7
:10383000C3B200935F4B1C685D685F4B20001A6841
:103840005B68290007F058FB02000B0020002900EC
:1038500006F0E4FC0022594B07F0E2F802000B00EE
:103860000020564907F048FB05F00AFEC3B22000CD
:1038700001240493394B022229001F703B00FFF7FB
:103880009FF94D4B3222186859683B00FFF798F9B1
:10389000324B02221C70454B186859682300FFF711
:1038A0008FF93068716823003222FFF789F93C00F4
:1038B0000F262500424B6235E15CEDB2711A2800FB
:1038C000C9B2FCF789FC013428000499FCF784FC98
:1038D000202CEED1FF2100981C4A6230C0B2131890
:1038E000843319701154E8E6364B1C78002C00D153
:1038F000A9E1354B354A1B781278134302D0FEF705
:1039000015FEDAE6324B1D78002D74D014AC192266
:103910002000304905F04AF9022D5FD120002E49E0
:1039200005F0A5F9DD23237423732000FDF778F853
:10393000C3E6C046984004409C4004405F08001025
:103940009F0900101C000010A40600102012001097
:103950008F0600108B060010630600106106001031
:1039600062060010D9050010D80500109B06001053
:1039700099060010AC060010580800103B0000101B
:10398000A6060010A7060010940600109C06001062
:1039900022000010A106001098060010D3060010A7
:1039A000F0C2000010C40000C8060010C0060010DD
:1039B0000000404000070010F806001000003040F2
:1039C000D40600109A060010A506001097060010F5
:1039D0009D0600101ABB0000A7BA0000032DA4D159
:1039E0002000D74905F043F9E02323732370013306
:1039F0002374237199E7D34AD34B12781B78002A9A
:103A00003FD00221D14A1170D14A1570002B34D019
:103A1000013B1A01CF4B9B18CF4A1868596812789E
:103A2000002A15D19C68DD6802000B0006F0F8FF43
:103A3000220006000F002B002000290006F0F0FFF6
:103A400002000B003000390006F0ACF802F034F947
:103A50000123C24C0C2223700023FFF7B1F8002190
:103A6000BF4B21701B788B4203D00A00B220FCF7B9
:103A700027FB0122B54B1A701FE600220C215F20A4
:103A8000F5E70092002B6FD1012208215F20FCF79F
:103A900017FB002612AC04222021200005F0A7F815
:103AA000B04B37001D782671B5420FD011AC04F031
:103AB000E3F9200014A904F087FA20220CAB9B182C
:103AC0001F7801320CAB9B18E5781E780022A04BC2
:103AD0001A7004F039F9AF231B01984200DBA248A9
:103AE000A24B984200DA1800A14BAF21C0180A235C
:103AF0008900584305F048FB2C23C0B25B424008C4
:103B0000181A12ABD870974B1C78002C00D1F7E232
:103B1000290012A8FEF77CFC12AD00226D212800BE
:103B2000FCF744FB01228A4B1A70002C00D134E3CD
:103B300039002800FEF76CFC0A21300005F020FB5C
:103B40003031E97030000A2105F094FA0A21C0B240
:103B500005F016FB3031A97001226D2112A8FCF787
:103B600025FBAFE5012300936A46774B12781B785B
:103B70000492009A934262D901220499521AD2B255
:103B800006920699724A1170009A9B1A013B714A7B
:103B90001B01D3181E685F689C68DD686E4B1B783C
:103BA000002B21D132003B003000390006F038FFF5
:103BB00022002B00089009912000290006F030FF18
:103BC00002000B000898099905F0ECFF02F074F868
:103BD0002200089009912B0030003900FCF7F0FF1B
:103BE000089E099F04000D00049B002B02D10122B6
:103BF0005A4B1A70082230003900069BFEF7E0FF8E
:103C00000022564B20001A7029000022002305F0E4
:103C1000B7FB002805D13B2220002900069BFEF7B8
:103C2000CFFF4F4B1B78002B09D0049B002B06D1F4
:103C30000122474BB22004991A70FCF741FA009B0D
:103C4000012B8FD139E54B4B1B78002B4AD0404ECE
:103C50002122210015A83470149404F0C8FF01211A
:103C600014A8FEF701FC050014A804F0F8FFC2B286
:103C7000002A10D103217F20FCF722FA01233370A0
:103C80003D4A11783D4AC900521810685168032214
:103C9000FEF796FF11E5102D22D92C000627103CC7
:103CA000E4B229001039611A794314AB185D03316D
:103CB00001340022C9B2E4B2FCF702FAA542F0D204
:103CC000DCE72900614303310022C9B20134FCF76B
:103CD000F7F9112CD2D014ABE05C0028F1D1CDE77C
:103CE0000625F8E7264B1C78002C02D0FFF72EFBA8
:103CF000E3E4244B1B78002B46D0154D21222100F4
:103D000015A82C70149404F072FF210014A8FEF77B
:103D1000ABFB31220CAB9B181C70113A0CAB9B18FF
:103D20001B7800220321002B05D15F20FCF7C8F986
:103D300001232B70A4E714A8FCF738FAF8E7C04673
:103D4000C0BA000089060010DC0500101B0000103E
:103D500061060010E0050010200000109E06001013
:103D6000DB0500108B060010EF0A0000340800008D
:103D7000CCF7FFFFA0060010281300102011001040
:103D80009F0600108D060010CD4B1B78002B00D134
:103D900057E1CC4B1B78002B01D0CB48C6E5CB4A72
:103DA00000931478002C44D11322202114A804F08D
:103DB0001EFF33220CAB9B1820211C705F230CAA22
:103DC000521813701D39012214A814E53B4300D08A
:103DD0008CE0BF4B0CA91A7833235B18002A0AD059
:103DE000BC4A1278002A06D10A0032212E2352182A
:103DF00013700CAA8B183022013B1A7014A8FCF720
:103E0000EBFD062414AD2878002800D00CE1B24B5D
:103E10001B78002B07D0069B002B04D10122190030
:103E2000B230FCF74DF9009B012B00D145E4012392
:103E300000936B46A54C1B78009A06932378934217
:103E4000F1D90123069A20219B1ADBB20893089A24
:103E5000A24B14A81A70132204F0C9FE33210022C9
:103E60000CAB5B181A70009923785B1A013B9C49D4
:103E7000DB00CB181E685F6833009742A6DA3C006F
:103E800000275E42A74101230493924B1B78002B2D
:103E90002ED033240CAAA4180322002394460CA984
:103EA0001E325218180061460133DBB2084202D1BB
:103EB0002021013C21700F25354028003030392861
:103EC00000D9273039073509013C294320703811C2
:103ED000070008000E00384301D101F0B9FB9442FD
:103EE000E0D8049B002B00D199E08EE00492CCE74F
:103EF000774B1D78002D58D00A220023300039005E
:103F000005F06CFA0A220C0005003900300000238D
:103F100005F064FA32210CAB5B1830321A702100C4
:103F20000A220023280005F059FA31210CAB5B1856
:103F300030321A7021000A220023280005F04EFAC0
:103F40000F0030212E2306000CAA5218137018AC53
:103F50002D3B32003A4301D101F07AFB21220CA91A
:103F600052189442BDD922781D002E2A0AD055221B
:103F7000524253430135DBB2EDB2552B02D8202318
:103F8000013C2370300039000A22002305F026FA94
:103F9000013C303200233000390022700A2205F043
:103FA0001DFA2B0006000F00D3E733240CABE418F6
:103FB00055222B00524253430135DBB2EDB2552B53
:103FC00002D82023013C2370300039000A2200234C
:103FD00005F004FA013C3032002330003900227031
:103FE0000A2205F0FBF9030006000F000B4301D184
:103FF00001F02EFB14AB9C42DAD8049B002B0ED0B0
:1040000021230CAA9B189C4203D8364914A804F01B
:104010002EFE2D23013C23703E4300D1EEE63149B4
:1040200014A804F024FEE9E62100089AFCF748F8F9
:104030002B78202B03D00634E4B20135E3E60334B9
:10404000FAE7294B1B78002B32D0284B1D78284BE0
:104050001B781D4300D052E4264BEEB21C78671942
:10406000FCF7CAFA874201DBFFF727FB34191B4B29
:10407000E4B220001E70FCF79BFA01340700E0B2A6
:10408000FCF796FA1C49C41B7918013C14AF2200B6
:10409000380004F08BFD00233200032138003B552B
:1040A000FCF784F8012D01D1FFF707FB0125D3E7C9
:1040B0001248FCF7B5FC01232B70FFF7FEFAC0464F
:1040C000A9060010AB060010D9BA00009319001021
:1040D00021000010910600109219001061060010D6
:1040E000981900108ABA0000A8060010A506001052
:1040F000970600109013001085000010F2BA00001F
:10410000B94B1B78002B02D0EC230CAA9376B74B4B
:104110001B78002B02D0DA230CAA9376B44B12AA98
:104120001B78002B05D0B34B1B7859424B41BD3354
:104130005370B14B1B78002B01D065331370AF4B1C
:104140001A7812AB002A22D048221A70AC4A127890
:10415000002A05D0AB4A1278312A01D8D8221A7029
:10416000A94BAA4A1B781278134300D1D4E4A84B78
:104170001B78002B00D0CFE40321A64B12AA1B789A
:1041800019409B084131313311705370C4E4A24A85
:104190001278002ADAD06822D7E7042220212800EA
:1041A00004F025FD984B2C711B78002B13D0994BF4
:1041B0001E783000FCF780F900286DD03000FCF745
:1041C00053F9964B0130C018035DFF2B03D02B55DC
:1041D0000134042CF8D18D4B914A1B78127813438B
:1041E00003D028008F4904F042FD8F4B1B78002B31
:1041F00008D01A208D4B19780CAB0131C9B2C01808
:10420000FEF706F97A4B1B78002B01D101F018FA62
:10421000874B1B78FF2B01D0D623AB70854C002237
:1042200020686168002305F0ABF8002847D1E3223D
:1042300012ABDA70804B814A1B7812781343804AA4
:10424000127813437F4A127813437F4A127813433C
:1042500012AA002B01D0E223D3707C4B1B78002BD9
:1042600005D07B4B1B78002B01D02E23D370794BCC
:104270001B78002B01D0A923D370774B77491B788B
:10428000002B05D1764B1B78002B00D164E47549D7
:10429000280004F0ECFC5FE42100212214AE15A8F4
:1042A000149404F0A4FC21003000FEF7DDF8335D27
:1042B000002B90D02B550134042CF8D18BE7002231
:1042C000A068E168002305F05BF80028AFD05F4BE1
:1042D0001B78002BAED0644A0CCA1343A7D1A9E7C0
:1042E00001331370FF230393FFF71AFA544B1C7822
:1042F000002C5ED05D4A13780133DBB213701D22AF
:104300003A70012B01D1FFF70BFA594E34687568EA
:10431000022B0CD1FCF79CFF22002B0005F042FC85
:10432000E02230607160534C534B120613E0032BB4
:104330001BD1FCF78DFF0022504B06F071FB0200F1
:104340000B002000290006F0D7FDE02230607160EC
:10435000484C4B4B12062068616805F023FC206036
:104360006160FCF725FAFFF7DBF9042B06D1FCF7B7
:104370006FFF0022414B06F053FBCDE7FCF768FFCF
:1043800002000B002000290006F0B6FD00223D4B84
:1043900005F044FFE022384B120605F03FFFFCF722
:1043A00007FA0122384B1A60254B009A1A70FF2336
:1043B00017E0224B1B780493002B00D1BFE02B4E5B
:1043C00033780133DBB23370022B5FD808D1FDF7AD
:1043D00075FBE02028490006FCF7EAF9FCF7C4FC6D
:1043E0001D233B70FFF79CF991060010A2060010F8
:1043F0009A060010200000108C0600109206001093
:10440000A1060010580800109F060010A00600101A
:104410008D06001028130010930600105F0800108E
:104420008F0600100BBB0000A806001090130010B0
:104430003B0000104013001099060010A706001062
:10444000A6060010940600109C060010A906001095
:104450002100001088060010A506001010BB000007
:104460009706001015BB0000B81900101F110010AE
:1044700080060010301300104D62503F00002040B5
:104480004D62603F000028401C000010FDF716FB45
:10449000FCF71EFD0020D149FCF78AF9FCF764FC0B
:1044A000E020CF490006FCF783F9FDF707FBFCF796
:1044B0000FFDFCF7CDFEFCF77BF907000D00FDF7C3
:1044C00087FB0022002338002900347004F05EFFCF
:1044D000002802D080231B06ED18E022C14C3800D2
:1044E0002900BF4B1206267804F050FF00280AD19D
:1044F000142E0AD8FCF726F9FCF724F923780133A7
:104500002370FFF70DF9142E0ED90CA8FCF710FC40
:104510001022B54914A8891804F048FB149815997D
:10452000169A179BFCF7EAF80122B04B1A6000229A
:10453000AF4B1A70AF4BFF321A70FFF7F1F8AE4B6A
:104540001E78002E6BD0AD4B1C780134E6B21E7085
:104550001D233B70012E01D1FFF7E2F8A84B1C6828
:104560005D68022E0CD1FCF773FE2B00220005F0D3
:1045700019FBA34B18605960A24B18685968F0E604
:10458000A14B1A685B6800920193032E10D1FCF7CF
:104590005FFE22002B0005F005FB994B1860596067
:1045A00000980199974B1A685B6805F0FBFAD8E60A
:1045B000162E20D80022F3071BD58023DB0504929A
:1045C0000593FCF745FE049A059B06F029FA2200A4
:1045D0002B0005F0E7FA8A4B18605960B01E07F00F
:1045E00071F8009A019B06F01BFA864B1A685B680B
:1045F000DBE7864BE3E7FCF72BFE009801992200EE
:104600002B0006F00DFA0022814B05F007FEFCF7A7
:10461000CFF80122754B1A60774B049AC6E67D4DA0
:104620002B78002B00D191E0744B1C780134E4B25C
:104630001C701D233B706B4B1A78002A41D1012C52
:1046400001D1FFF76DF86F49086849680090019142
:10465000022C0AD1FCF7FCFD6F4B186059606F4BC0
:1046600018605960009801997BE6222C24D8FCF749
:10467000EFFD6A4D06000F0002000B002868696814
:1046800004F098FE002801D02E606F60624D320069
:10469000286869683B0004F079FE002801D02E608C
:1046A0006F60A01E07F00EF8574B1A685B6806F0A3
:1046B000B7F9009A019B78E750490A7001221A70F5
:1046C000D0E7012C01D1FFF72BF8212C2ED8534B2A
:1046D0001C685D68FCF7BCFD02000B00200029008F
:1046E00006F00AFC4C4B06001A685B680F002000BD
:1046F000290006F001FC02000B003000390005F033
:104700008DFD0022464B06F08BF901F0BBF93B4BC7
:10471000444C1D7804F0B4FE6419023C2070681EFD
:1047200006F0D0FF384B1A685B685CE70CA8FCF712
:10473000FFFA0CA8FCF7FCFA01232C4A2E70136038
:10474000FF223A70384A1370FEF7EAFF0A20374B0F
:1047500003211B78584303F087FFFDF761F9387098
:10476000FEF7DEFF324B1C78002C00D13BE11D2808
:1047700002D0122800D0A5E02E4B1B780393002B0B
:1047800060D02D4B1D782800FBF76EFE040028003A
:10479000FCF786F9294F380004F061FA0500202063
:1047A000FBF762FE264E021B611E601989198019F3
:1047B00004F03FFAFE2300253355380004F04FFA89
:1047C000A84206D97A5D631CF3185A550135072DA6
:1047D000F3D10022164B1A70FEF7D7FF0000F0BF8E
:1047E0004D62503FAD06001080BC00001C00001060
:1047F000A7060010AC060010940600101F11001050
:1048000080060010C006001078060010000010405E
:10481000000008409C060010F80600100007001079
:1048200000002E40D40600109B060010220000104D
:104830008F0600109F06001028130010630600105A
:104840005F080010D44B1B78002BC2D0D34B1C78D0
:104850002000FBF7ADFE01340700E0B2FBF7A8FE35
:10486000CF4E0500300004F0FAF9C4B2FBF7B6FEF3
:10487000691E421BCB4DE01901324919401904F061
:10488000D8F97B19180022003100049304F08EF946
:10489000C54B1B78002B9CD0C44E3378FC1800937A
:1048A000FBF79CFE009B6119C21B0134D2186019F2
:1048B00004F0BFF90A2233780499CA54BA4B039A18
:1048C0001A7086E7012804D10F22B94B1A70FEF73F
:1048D0005CFF022809D1B74A13780B2B01D9FEF7E8
:1048E00054FF01331370FEF750FF042809D1B04A7A
:1048F0001378002B01D1FEF748FF013B1370FEF740
:1049000044FF052804D10822A94B1A70FEF73DFF89
:10491000062809D1A64A13780E2B01D9FEF735FFD8
:1049200001331370FEF731FF072804D10022A04B9A
:104930001A70FEF72AFF082809D19E4A1378002B27
:1049400001D1FEF722FF013B1370FEF71EFF18286E
:1049500009D1964A1378002B01D1FEF716FF013BCF
:104960001370FEF712FF19280DD1904C8C48257852
:1049700004F075F9854201D3FEF707FF2378013370
:104980002370FEF702FF21280ED1884C20780028E2
:1049900001D1FEF7FAFE0138C0B2FDF729FD2378F8
:1049A000013B2370FEF7F1FE7D4C200004F057F927
:1049B000814B1A780723002A00D10B33984201D388
:1049C000FEF7E3FE7A4B19787A4B20311B781B01F6
:1049D000C918764BC9B21A78501C18702000FBF722
:1049E0007DFEFEF7D2FE754D2A78002A47D01E289C
:1049F00002D12C70FEF7C9FE12280BD1704B1A7829
:104A0000704BD2009B1818685968FBF7D1FE2C70C8
:104A1000FEF7BBFE082809D1694A1378002B01D1A3
:104A2000FEF7B3FE013B1370FEF7AFFE022809D17B
:104A3000634A1378222B01D9FEF7A7FE01331370C6
:104A4000FEF7A3FE09280AD15D4A1378042B03D987
:104A5000053B1370FEF799FE1470FEF796FE0328CF
:104A600001D0FEF792FE564A13781E2B03D8053369
:104A70001370FEF78AFE23231370FEF786FE524B57
:104A80001C78002C02D01A70FEF77FFE4F4E337850
:104A9000002B58D04E4D2B78002B0ED0021FD1B2D8
:104AA00005290AD8591E06234B439B18494A9B00E7
:104AB0009B5898472C70FEF768FE474B1B78002BDD
:104AC00027D00438C4B2052C1ED83222100060430F
:104AD000424D434B2900C01804F068F82A78414B36
:104AE000A400FF2A0BD000223F481B19A95CFF2914
:104AF0000AD0415C99540132042AF7D104E02D22F6
:104B00001A5500221B195A700022334B1A70FEF7F7
:104B10003CFE364B1B78002B11D00438C1B205295E
:104B200006D8322251432E4809182C4804F03EF88A
:104B3000FCF72AFF00222D4B1A70FEF726FEFCF729
:104B400085FEFEF722FE2A4D2B78002B00D1E3E0F4
:104B500003001D3B274E012B01D912280BD1002346
:104B60002B70FCF711FF3078FCF7A4FE3078FCF7CF
:104B7000A1FEFEF70AFE3478182850D11E4F3D786A
:104B8000022D3DD12000FBF76FFC1C4B1B5CFD2B65
:104B9000E9D0013D41E0C046A80600109013001086
:104BA00063060010850000109606001062060010D3
:104BB000D8050010D90500109F06001098060010B7
:104BC000D3060010F0C200009B0600109A060010E9
:104BD0009D060010A0C40000A50600103B000010B8
:104BE0000807001023000010C8C20000970600103C
:104BF000A006001028130010600600105F080010C7
:104C0000012DB0D92000FBF72FFCD24B5B191B18EC
:104C1000023B1B78FD2BBCD1023D3D70A3E7192858
:104C200015D1CD4B1B78002B70D12000FBF71CFC5D
:104C3000CA4FC84B3D781B185B5DFD2B01D1023577
:104C4000EBE7FBF727FCA8428DD90135E5E72128E2
:104C500040D1C24D2F78002F85D07B1EDBB2009350
:104C6000012F32D02000FBF7FFFBBA4BDF193F18B2
:104C7000023F3B78FD2B28D120000099FBF736FF3F
:104C8000297830780239C9B2FBF730FF2B78013B25
:104C90002B702B78013BDBB22B70002B00D062E72E
:104CA00037783800FBF7E0FBAA4C235CFF2B00D1E0
:104CB00059E7012338002B70FBF7D6FB235CFD2B53
:104CC00000D050E7FB3B2B704DE720000099FBF72D
:104CD0000DFFDEE70B2808D1A04B1A78511C197084
:104CE00012212000FBF7AEFD3DE726280ED19C4B9C
:104CF0001C709C4B1A789C4B1A709C4B1A789C4BDE
:104D00001A7001229B4B1A700023DCE7934B1A7830
:104D1000511C19700100E4E7974C2378002B00D157
:104D20006EE1964C23780093002B0BD00438C3B26D
:104D3000052B03D8924B8000C3589847002323705B
:104D4000FEF723FD8F4B1B78002B31D08E4B1D7847
:104D50002800FBF789FB04002800FBF7A1FE8B4F1E
:104D6000380003F07CFF05002020FBF77DFB794E27
:104D7000021B611E60198919801903F05AFFFE2376
:104D8000009D3355380003F06AFF854206D27A5DF4
:104D9000631CF3185A550135072DF3D10023794AC6
:104DA0001370FEF79BFA0122794B1A60FEF7EDFCB7
:104DB000784B1B78002B29D00438C4B2052C00D9BD
:104DC000A2E6A022520010006043734B614DC01850
:104DD000290003F0EBFE1F20FBF746FB2B5C6F491D
:104DE000A400FF2B0CD00123013C0C192818C25C35
:104DF000FF2A00D188E6E2540133052BF7D183E680
:104E00002D230B5500230C1963707DE6644B197834
:104E100000290BD00438C1B2052900D988E6A022A8
:104E2000520051435C4809184A487FE61E2803D1C6
:104E300001232370FEF7A9FC08280CD14B4B524AE2
:104E400019701378032B03D9043B1370FEF79DFCF4
:104E50001170FEF79AFC02280CD10122434B1A7004
:104E6000494A13781B2B01D9FEF78FFC04331370CA
:104E7000FEF78BFC042812D1434A1378002B01D093
:104E8000013B1370002337490B701378DB439B07FA
:104E900001D0FEF77AFC01230B70FEF776FC0628A2
:104EA00013D1394A13781E2B01D801331370012115
:104EB0002C4B19701178032208001040114201D0C8
:104EC000FEF763FC1870FEF760FC122801D005287D
:104ED00068D101232B70274B2B4F1E783C78002E76
:104EE00021D01F4B1D4D18781F4BFD211A781D4BEB
:104EF00038701A701E4B1A781C4B1A702A78531C83
:104F00002B70FBF79FFC2A782100531C38782B70FC
:104F1000FBF798FC0023174A1370FCF735FDFEF7EA
:104F200015FAFEF732FC2000FBF7C6FA071E05D083
:104F30003000FBF7B1FE2E70FEF727FCFBF7AAFA54
:104F4000FF2800D13800054B18702000FCF7B2FC98
:104F5000FEF71BFC5F0800108C06001060060010B6
:104F6000D006001029130010D10600102A130010DB
:104F7000D2060010A20600109F060010A306001023
:104F8000E8C400009006001028130010630600100B
:104F90001C000010A50600109F0900106D000010F5
:104FA000970600101D2811D1CD4B1878FBF75CFA3D
:104FB000CC4B1B5CFE2B04D10020FBF76DFEFEF7F3
:104FC000E4FB0120FBF768FEFEF7DFFB212807D199
:104FD000C34B1878FBF764FDFCF7D6FCFEF7D5FB56
:104FE000252804D10122C04B1A70FEF7CEFB2628DB
:104FF00001D0FEF7CAFB0122BC4B1A70FEF7C5FBBD
:10500000BB490A78002A00D1C1E01E280DD1B94A57
:105010000B701078B84A1070B14C2078FCF74AFC3D
:105020002078FCF747FCFEF7B0FB1D2809D10123CF
:105030002B70FBF72FFAFF2800D10020AF4B187020
:10504000EAE7122801D00B2812D1AD4B12201B78B1
:10505000002B00D098E00120FBF706FA0400202086
:10506000FBF702FA9F490200601803F0E2FDD3E764
:10507000212825D12038FBF7F7F904002020FBF781
:10508000F3F99F4D02002E78964B002E14D0661E29
:105090009E19012C07D931000232A01E121B1818CC
:1050A00003F084FDB8E7013219193000121B03F038
:1050B0007DFD00232B70AFE7021B19191800EFE7E5
:1050C0000A2823D88E4E202033780093FBF7CCF9A2
:1050D000009B0400834D002B0CD00120FBF7C4F98A
:1050E0000134461E221AA919281803F0A2FD3B78A4
:1050F000AB5591E702002900824803F09AFD3B7806
:105100002B70FF236B70FE3B337085E70F283BD875
:105110000120FBF7A9F900900220FBF7A5F9040094
:105120002020FBF7A1F90700009B6E4DE31A0393C3
:105130005B19020029001800049303F07AFD039A1A
:105140006119280003F032FD009B6100DE19361B57
:10515000C91A321B4919601903F028FD039B32005C
:10516000581E0499401903F021FDA61EBA1C601EAA
:10517000121B7119401903F05CFD0022624B1B7871
:10518000AB555F4B1A7047E7FBF778FB44E75F4D81
:105190002B78002B00D1FFE05D4C2378002B0BD047
:1051A0000438C3B2052B03D85A4B8000C358984724
:1051B00000232370FEF7E9FA1E2803D10123237090
:1051C000FEF7E3FA212847D1534B1B78002B3FD041
:1051D000524B1B78002B29D0FBF7A4F9FA220023AD
:1051E000920007000E0004F0F9F80B0005000C0017
:1051F000034303D1FBF7AAF9FEF7C7FA38003100E1
:105200006422002304F0EAF8D3B20A930023642254
:105210000B9328000023210004F004F90A9B0B9C47
:10522000C0186141FBF744FBFEF7AFFAFBF77AF9D0
:105230003B4B10221C7800239C4200D1063A04F01C
:10524000CDF80B000343D5D0FBF732FBFEF79DFAF8
:10525000FBF768F9FEF799FA1F2806D1314B1B7846
:10526000022BC7D9FCF7BBFFC4E7132817D1FBF704
:1052700059F904F05FF900F01FFD284B00221B785C
:10528000002B0AD1284B05F0CBFB04F017F9FBF7F4
:105290000FFBFBF75BF9FEF778FA244BF3E72028C6
:1052A00006D1204B1B78012BA4D9FCF7B2FFA1E754
:1052B000252809D1FBF736F91D4B03C3FBF7F8FA94
:1052C000FBF744F9FEF761FA262833D1184B18682A
:1052D0005968FBF7EDFAFBF739F9FEF756FAC046C5
:1052E000281300105F080010A50600109706001094
:1052F0008D0600108A060010890600106006001056
:105300008E06001061080010AC060010A9060010FF
:10531000AB0600104CC500009219001021000010CF
:1053200091060010931900100000F03F0000244087
:10533000B819001016281DD1CA4C2378012B01D9A9
:10534000FCF767FFFBF7D2FA2378022B01D9FCF7B1
:1053500046FFFCF7D9FDC44B64201B78002B00D01E
:10536000C2480021FBF7A4FAFBF7E8FAFBF7EEF8D6
:10537000FEF70BFA122801D9FEF707FABC4B8000A2
:10538000C35898473B780A2B01D8FEF7FEF9122B39
:1053900001D1FEF7FAF92DE7B64F3B78002B3FD04D
:1053A0001E2803D100233B70FEF7EFF9132804D128
:1053B0001238FBF7ADFBFEF7E8F90F2804D10E38E1
:1053C000FBF7F4FAFEF7E1F9142804D10F38FBF7E4
:1053D0009FFBFEF7DAF9092804D10438FBF7E6FA57
:1053E000FEF7D3F9152804D10B38FBF791FBFEF734
:1053F000CCF9082804D10230FBF7D8FAFEF7C5F93A
:10540000162804D10238FBF783FBFEF7BEF9072804
:1054100001D0FEF7BAF90D30FBF7C8FAFEF7B5F97F
:10542000954A1378002B00D1D6E0944B1B78002BC3
:105430001ED00438C4B2052C01D9FFF765FB8022C9
:105440008F4B904D20022900C018520003F0AEFB94
:1054500000232021A0008C4C2418EA5C21700A2A29
:1054600000D0227001330134042BF6D1FFF74CFB3E
:10547000864C217800290FD00438C0B2052807D8FF
:10548000802201027E48520009187E4803F08EFBFC
:1054900000232370FEF779F91E2802D11170FEF760
:1054A00074F9082809D17A4A1378002B01D1FEF744
:1054B0006CF9013B1370FEF768F902280BD1FBF77A
:1054C0009BF8734D2C780134844201DBFEF75DF9C3
:1054D0002C70FEF75AF909280AD16D4A1378042B6B
:1054E00003D9053B1370FEF750F91170FEF74DF923
:1054F00003280ED1FBF780F8654D2C78A31D83425D
:1055000003DA05342C70FEF740F901382870FEF7F5
:105510003CF9122803D1FBF70FFBFEF736F90F28F1
:1055200006D1FBF709FB01225A4B1A70FEF72DF941
:10553000212801D00D281BD1554E34782000FBF7CF
:1055400037F801340500E0B2FBF732F80400FBF74E
:1055500045F8021B4B482118281803F027FB337825
:10556000002B01D1FEF711F9013B3370FEF70DF965
:105570000E281CD1FBF740F8012801D8FEF705F9E9
:10558000434B18780130C0B2FBF712F83D4D0400D0
:105590002B5C002B01D1FEF7F8F8FBF71FF8021B7C
:1055A000601E6119401903F001FBFEF7EEF80C28AC
:1055B00000D015E5364B1878FAF7FAFF0400FBF730
:1055C0000DF8304D021B601C6119401903F031FBCE
:1055D0000A232B55FEF7D9F8072803D1012333708E
:1055E000FEF7D3F808280AD12B4A2C4814781370F8
:1055F00001220A702A4A04701370FEF7C6F80928BF
:1056000008D1254A254910781370012308702370AA
:10561000FEF7BBF8042803D101232B70FEF7B5F881
:10562000052805D101233B70FBF7B6FAFEF7ADF86C
:10563000062801D0FEF7A9F801231370FEF7A5F89C
:10564000184B1B78002B01D0FEF7E8FDFEF73FFE5C
:10565000049B00260027002B01D0FEF7D1FCFEF7AB
:10566000CDFBC04693190010210000101027000048
:1056700000C50000A4060010A8060010A506001032
:10568000911300108500001085010010970600108E
:105690009013001096060010890600108A0600106C
:1056A000281300108D060010F8B54E4657464546A3
:1056B000DE46A34BE0B54E00804689468A46760812
:1056C0009E421CDD9F4B9E4209DC06D05346002BB8
:1056D00000DCBAE09C4B9D4A09E00028F6D0424627
:1056E0004B464046494604F05DFA03000A001800A4
:1056F0001100F0BCBB46B246A946A046F8BD944B8B
:105700009E4200DDA4E0934B9E4200DC8FE001232B
:105710005B429B4642464B464046494605F080F96F
:1057200002000B0006000F0005F07AF904000D00DE
:10573000894A8A4B05F074F9894A8A4B04F032FA97
:1057400022002B0005F06CF9874A884B04F02AFAF6
:1057500022002B0005F064F9854A864B04F022FAFA
:1057600022002B0005F05CF9834A844B04F01AFAFE
:1057700022002B0005F054F9814A824B04F012FA02
:1057800032003B0005F04CF97F4A804B06000F00C9
:105790002000290005F044F97D4A7E4B05F0ACFB62
:1057A00022002B0005F03CF97B4A7C4B05F0A4FB62
:1057B00022002B0005F034F9794A7A4B05F09CFB66
:1057C00022002B0005F02CF9774A784B05F094FB6A
:1057D00022002B0005F024F90B005946020001318C
:1057E0005CD059463000CC00390004F0DBF9424669
:1057F0004B4605F015F96E4D6E4B2D191C1922689C
:10580000636805F079FB42464B4605F075FB0200E4
:105810000B002868696805F06FFB030050460A001A
:10582000002800DB63E7802212068A185FE7624ADD
:10583000624B04F0B7F90022614B03F0BBFD002876
:1058400000D164E743464A4651E73F4B5D4A4EE785
:1058500000F014F95C4B04000D009E422FDC5B4B02
:105860009E4255DC02000B0004F09CF90022544BD0
:1058700005F042FB802306000F000022DB0520001C
:10588000290004F08FF90B0002003900300004F009
:10589000C5FC0023804689469B463BE73000390023
:1058A00004F080F942464B4605F0BAF802000B00BE
:1058B0004046494605F020FB03000A0017E7444B29
:1058C0009E421ADC0022434B05F016FB0022060024
:1058D0000F00404B2000290005F0A2F80022384BB1
:1058E00004F060F90B0002003900300004F096FC6F
:1058F0000223804689469B460CE70B00020036498E
:10590000002004F08BFC0323804689469B4601E778
:1059100000222B4B05F0F0FA002206000F00284B66
:105920002000290004F03EF90B000200390030008D
:1059300004F074FC0123804689469B46EAE6C04693
:10594000FFFF0F440000F07F182D4454FB21F93F66
:10595000FFFFDB3FFFFF1F3E11DA22E33AAD903F2E
:10596000EB0D76244B7BA93F513DD0A0660DB13F96
:105970006E204CC5CD45B73FFF8300922449C23FFE
:105980000D5555555555D53F2F6C6A2C44B4A2BFC3
:105990009AFDDE522DDEAD3F6D9A74AFF2B0B33F8B
:1059A000711623FEC671BC3FC4EB98999999C93F03
:1059B00068C5000088C500009C7500883CE4377EFF
:1059C0000000F03FFB21F9BFFFFFF23FFFFFE53F83
:1059D000FF7F03400000F83F0000F0BFD0B5254A2C
:1059E0004B0086B05B08934222DD234A934209DDD7
:1059F00002000B0005F080FA02000B0010001900F5
:105A000006B0D0BD02AA00F02BFD03231840049A73
:105A1000059B012813D0022822D0002819D0029813
:105A200003990124009401F075FD02000B00E5E7E5
:105A30000022002300F0F4FF02000B00DEE70090DC
:105A40000298039901F066FD80231B060200CB1823
:105A5000D4E70298039900F0E3FF02000B00CDE7C2
:105A60000298039900F0DCFF80231B060200CB188C
:105A7000C4E7C046FB21E93FFFFFEF7F4B00590819
:105A80007047C046F8B504004A000B0008002649DC
:105A9000520D5118270013291ADC002912DB234A62
:105AA00026000A41100018401D00204307D0802026
:105AB000000308410024C018904326000500300070
:105AC0002900F8BDDB0FD8074B1C28D00024F4E7D1
:105AD00033290DDD802226001D00D2009142EED137
:105AE00022002000190004F05DF806000D00E6E732
:105AF0000F4D2600AC46012562446D42D540AC46B0
:105B000062461D002242DAD03322511A323A8A40CC
:105B10001419A74200D9581C63469C43CDE7054B96
:105B200000241843C9E7C04601FCFFFFFFFF0F0038
:105B3000EDFBFFFF0000F03FD0B5264A4B0086B0DA
:105B40005B08934222DD244A934209DD02000B00E8
:105B500005F0D2F902000B001000190006B0D0BD0C
:105B600002AA00F07DFC03231840049A059B01283B
:105B700015D0022823D0002818D00298039900F0ED
:105B80004FFF80231B060200CB18E5E7002300220D
:105B90000093002301F0BEFC02000B00DCE702983A
:105BA000039900F03DFF02000B00D5E701240298A5
:105BB0000399009401F0AEFC02000B00CCE7012435
:105BC00002980399009401F0A5FC80231B060200B3
:105BD000CB18C1E7FB21E93FFFFFEF7FF8B50400D9
:105BE0000D0000F091F806000F002000290001F0E0
:105BF00079FD00280FD0200029000F4A0F4B03F039
:105C0000D9FB00280AD1200029000D4A0D4B03F0D2
:105C1000BDFB002809D130003900F8BD05F000FFB8
:105C200022230026084F0360F5E705F0F9FE222342
:105C3000002600270360EEE7EF39FAFE422E864089
:105C400051302DD5104987C00000F07FF8B5040011
:105C50000D0000F00BFA220006000F002B002000C0
:105C6000290005F0DBFC002815D1002200232000CC
:105C7000290003F09FFB00280DD100220023200003
:105C8000290003F07DFB002808D005F0C9FE22237F
:105C90000026074F036030003900F8BD05F0C0FE54
:105CA00021230360034801F0C3FD06000F00F2E763
:105CB0000000F0FFA8C50000F8B504000D0000F0DA
:105CC000D7FD220006000F002B002000290005F060
:105CD000A5FC002807D1002200232000290003F0A2
:105CE00055FB002802D130003900F8BD05F098FEC0
:105CF00021230022036000231000190004F08EFA13
:105D000006000F00EFE7C046F0B5D64600B54B00E1
:105D10000E00CC0FB549070088B05B088B420FD945
:105D2000B3498B4229D93203120B024300D040E120
:105D300005003300002C00D11CE10025002319E1EF
:105D4000AC4A934200D91BE1AB4A934200D9BCE074
:105D5000AA4AAB4B310003F025FF0022A94B03F008
:105D600029FB002800D1B0E00022A64B380031000A
:105D700003F018FF05000B00FCE03100A24AA34B22
:105D800003F018FB002800D016E138003100A04ACB
:105D9000A04B03F0FBFA002800D021E19E48E4006C
:105DA00004199E4A9E4B3800310004F039FE2268E7
:105DB000636803F0F7FE05F04FFC824605F082FCB5
:105DC000984A994B04000D0004F02AFE02000B00D3
:105DD0003800310005F090F8944A02900391944BFA
:105DE0002000290004F01CFE04900591049A059BF4
:105DF0000298039905F080F802000B0007000E00DE
:105E00000090019104F00CFE04000D00894A8A4BB9
:105E100004F006FE894A8A4B05F06EF822002B003A
:105E200004F0FEFD874A884B03F0BCFE22002B00E5
:105E300004F0F6FD854A864B05F05EF822002B0043
:105E400004F0EEFD834A844B03F0ACFE22002B00ED
:105E500004F0E6FD0B0002000098019905F04CF8F3
:105E6000534604000D0006940795002B61D00200F4
:105E70000B000098019904F0D3FD0F00802106006B
:105E800022002B000020C90505F036F802000B00A7
:105E90003000390004F0C2F902000B0004980599A3
:105EA00005F02AF8029A039B05F026F80B00020081
:105EB0005449002005F020F8684B9A4500DA81E04B
:105EC000544624050500631854E03A0033003800B6
:105ED000310004F0A5FD04000D00564A564B04F0B5
:105EE0009FFD564A564B05F007F822002B0004F0A0
:105EF00097FD544A544B03F055FE22002B0004F04A
:105F00008FFD524A524B04F0F7FF22002B0004F0A1
:105F100087FD504A504B03F045FE22002B0004F051
:105F20007FFD02000B003800310004F0E5FF069011
:105F30000791069A079B3800310004F071FD802319
:105F40000D000400069807990022DB0504F0D4FF39
:105F500002000B002000290004F060F93A00330031
:105F600004F0CAFF0B0002002649002004F0C4FF21
:105F700005000B002800190008B080BCBA46F0BD2F
:105F8000374A934200D909E7364BE5005B191A6896
:105F90005B68310004F0B0FF029003910120324BA6
:105FA000001B5B191A685B6804920593031B9A46F1
:105FB0001CE702003300D9E6002001F08BFB05004E
:105FC0000B00D7E7FA24A4005444240563181900F1
:105FD000B82300225B0404F023FD05000B00C9E791
:105FE000002001F06FFB05000B00C3E7412E864047
:105FF000FFFFEF7F422ED63FFFFFEF3D9C750088ED
:106000003CE4377E0000F03FEF39FAFE422E864036
:1060100051302DD5104987C0B0C50000FE822B65D8
:106020004715F73F0000E0FE422EE63F763C79350B
:10603000EF39EA3DD0A4BE726937663EF16BD2C536
:1060400041BDBB3E2CDE25AF6A56113F93BDBE1647
:106050006CC1663F3E5555555555C53F03FCFFFF86
:10606000B1A2F03FC0C50000D0C50000F0B5D646D3
:106070004F4646468022C0B50B0088B0520391427D
:1060800055DA4A005208024300D1EBE0002900DA59
:1060900023E1D64B002204F0C3FC3625D44C0B0080
:1060A0006D42A34247DCD34C1A151B031B0B9846C9
:1060B000A4468024D04B640343442340CF4C624425
:1060C00052195C4045461B1599462543CB4B290088
:1060D0009144002204F010FF434602331B030600E4
:1060E0000F0000221B0B022B2FDC002303F048F9CA
:1060F000002800D1BDE04B46002B00D148E14846C6
:1061000005F0E0FABE4ABF4B04000D0004F088FC25
:10611000BD4A06000F0020002900BC4B04F080FCA3
:1061200002000B003000390003F03CFD07E0B04CEA
:106130000025A342B7DD02000B0003F033FD08B0D9
:10614000E0BCBA46B146A846F0BD8023DB0503F0AB
:1061500029FD02000B003000390004F05FF8040054
:1061600048460D0005F0AEFA22002B000490059180
:10617000200029000294039504F052FCA44B020075
:1061800043449A460B000090019104F049FC04003E
:106190000D00A04AA04B04F043FCA04AA04B03F022
:1061A00001FD22002B0004F03BFC9E4A9E4B03F0B5
:1061B000F9FC22002B0004F033FC9C4A9C4B03F0BA
:1061C000F1FC009A019B04F02BFC9A4A009001918B
:1061D000994B2000290004F023FC984A984B03F0C7
:1061E000E1FC22002B0004F01BFC964A964B03F0C6
:1061F000D9FC22002B0004F013FC0B0002000098D5
:10620000019903F0CFFC0D004146904B04005B1A4E
:1062100051460B43002B52DD00228D4B30003900DC
:1062200004F0FEFB3B00320004F0FAFB4B4600900A
:106230000191002B59D102000B002000290003F02E
:10624000B1FC029A039B04F0EBFB02000B000098E8
:10625000019904F051FE02000B003000390004F0F7
:106260004BFE6CE70022002300207A4903F0D6FFA2
:1062700065E7794A794B3000390004F0D1FB020020
:106280000B000020724904F037FE320004000D00BC
:106290003B003000390004F0C3FB0B000200290072
:1062A000200004F0BDFB4B4604000D00002B4DD137
:1062B00002000B003000390004F01EFE3FE74B46A1
:1062C000002B68D122002B003000390004F014FEAE
:1062D000029A039B04F0A4FBBDE7020004F00CFE4D
:1062E0000022002303F09AFF29E7454A454B049812
:1062F000059904F095FB009A019B069007912000F8
:10630000290003F04FFC029A039B04F089FB3E4AEC
:1063100004000D00049805993C4B04F081FB020039
:106320000B002000290003F03DFC02000B00009848
:10633000019904F0E1FD32003B0004F0DDFD0200B4
:106340000B000698079904F0D7FDF8E6484605F0DB
:10635000B9F92B4A2B4B0090019104F061FB2A4ABA
:106360000290039100980199284B04F059FB020018
:106370000B002000290004F0BFFD32003B0004F0B8
:10638000BBFD02000B000298039904F0B5FDD6E6B0
:1063900000200021D3E61A4A1A4B0498059904F00C
:1063A0003FFB2200009001912B003000390004F0E7
:1063B000A3FD029A039B04F033FB134A04000D0073
:1063C00004980599114B04F02BFB02000B002000F0
:1063D000290004F091FD32003B0004F08DFD020025
:1063E0000B000098019904F087FDA8E600005043D7
:1063F000FFFFEF7F01FCFFFF645F09000000F03F3B
:106400000000E0FE422EE63F763C7935EF39EA3D6A
:1064100086EBF9FF44523EDF12F1C23FDE03CB961A
:106420006446C73F599322942449D23F935555550A
:106430005555E53F9FC678D0099AC33FAF788E1D6A
:10644000C571CC3F04FA97999999D93F51B8060084
:106450000000E03F000050C3555555555555D53FF8
:10646000F0B54E465746DE464546E0B5DF4B4E009A
:10647000170089468FB076089E4200DC8BE0DC4B2B
:106480009E4228DCDB4A002900DC90E1DA4B04F074
:1064900033FDD94B04000D009E4200D191E0D74A54
:1064A000D74B04F029FD02000B0020003A607B600E
:1064B000290004F021FDD24BD04A04F01DFD012338
:1064C0009846B860F96040460FB0F0BCBB46B24693
:1064D000A946A046F0BDCB4B9E4200DC8DE0CA4BE6
:1064E0009E4263DCC94932158846904443461B05E9
:1064F000F51A2900040005F0AFF805F0E3F80200F2
:106500000B00200029000892099304F0F5FC0022FA
:10651000BF4B04F085FA0D00040005F09DF806005D
:1065200005F0D0F802000B00200029000A920B931E
:1065300004F0E2FC0022B64B04F072FA00220023C1
:106540000C900D9102F01CFF002800D103E13300F4
:106550005A1E93410133AF4A39000192022208A822
:106560000092424600F074FB4B468046002BAADAAC
:1065700080200006844679683A6861440B00F96817
:106580003A607B6061440B00BA68BA60FB604346C6
:106590005B42984697E702000B003A607B6000235D
:1065A0000022BA60FB60002398468CE70B000200D3
:1065B00004F0A2FC0023B860F96098463860796066
:1065C00081E7D3228E4B520504F096FC924A934BFE
:1065D00004000D0004F090FC02000B0020003A6063
:1065E0007B60290004F088FC8C4B8B4A04F084FC0F
:1065F0000123B860F960984665E7FFF73FFA884ADB
:10660000884B04000D0004F00BFA0022864B03F0C7
:10661000C9FA05F021F8804605F054F8754A764B22
:106620000490059104F0FCF902000B002000290001
:1066300004F062FC724B02900391049805996F4A32
:1066400004F0EEF9434604000D001F2B36DC774AB8
:10665000013B9B009B58B34230D002980399220023
:106660002B0004F049FC82468B4652465B463A605A
:106670007B600298039952465B4604F03DFC220081
:106680002B0004F039FC030008001A001900030075
:10669000BA60FB604B46002B00DB14E780238024AC
:1066A0001B069C464346554624065C4460445B42B8
:1066B00098463D607C60B960F86004E72B00029862
:1066C0000399220004F018FC4B0036155B0D82463E
:1066D0008B46F31A102BC8DD04980599D322484B3A
:1066E000520504F09DF904000D0002000B00029811
:1066F000039904F001FC02000B0002980399069232
:10670000079304F0F9FB22002B0004F0F5FB0400D2
:106710000D0004980599404A404B04F081F922008D
:106720002B0004F0E9FB0B00020004000D000698AA
:10673000079904F0E1FB4B005B0D82468B46F61A8D
:10674000312E0ADC02000B003A607B60069A079B40
:10675000029203938DE70323FDE6B822049805997E
:106760002E4B920504F05CF904000D0002000B00B2
:106770000698079904F0C0FB02000B0006980799E1
:106780000292039304F0B8FB22002B0004F0B4FB48
:1067900004000D0004980599254A264B04F040F9A1
:1067A00022002B0004F0A8FB04000D0055E7124B5B
:1067B00003F0F8F9104B04000D009E423CD00F4A44
:1067C0000F4B03F0EFF902000B0020003A607B60F2
:1067D000290004F091FB094A094B03F0E3F9012376
:1067E0005B429846B860F9606DE6C046FB21E93F20
:1067F0007BD9024000004054FB21F93F3163621A0B
:1068000061B4D03DFB213941FFFFEF7FEAFBFFFF81
:106810000000704160C600007370032E8A19A33B0C
:1068200083C8C96D305FE43F0000E03FE0C5000071
:10683000C14920259A837B39D3220A4B520503F0A4
:10684000B1F9094A094B04000D0003F0ABF902004D
:106850000B0020003A607B60290004F04DFB024AE7
:10686000024BBAE761B4D03D7370032E8A19A33B83
:10687000F8B5684BCE4647460500020018000C00EC
:1068800080B50840984200D1A0E0002969DD0815D4
:1068900000D177E0604B0903C4188023090B5B0328
:1068A0001943C30703D4D30F49005918520063108A
:1068B00098464B00D10F5B180021802016248C468F
:1068C000520080030D189D4202DC29185B1B844492
:1068D000D50F5B00013CEB1852004008002CF1D1B1
:1068E0000020814680202026000609E08B425ED0F1
:1068F000D50F5B00013E5B1952004008002E16D0F8
:1069000005198B42F2DD0F002C18002D4BDB5B1AB2
:10691000AA42894149425B1A521BD50F5B00013ED6
:10692000814439005B1952004008002EE8D113431E
:1069300045D14B465E0863465910384B994663462D
:106940004944DB0702D580231B061E434346180536
:10695000431835001C0028002100C0BCB946B046D1
:10696000F8BD4B005B082B43F5D0002000293AD13D
:10697000D30A190015385205002BF9D0802464037E
:10698000234241D1802300245B03490025000134C8
:106990001942FAD020260B001100A240361BF1400C
:1069A000401B194376E7E743FF0FCF19AFE7954246
:1069B0009ED82C18002DF6DB1F000023ACE74B46B9
:1069C00001331DD04E4601367608B4E72A000B008D
:1069D0002800210004F024F82A00230003F0E2F844
:1069E00005000C00B7E72A000B002800210004F086
:1069F00083FA02000B0003F011FC05000C00AAE76B
:106A000001239946CC4496E70125110020266D42CA
:106A1000C5E7C0460000F07F01FCFFFF0000E03F3B
:106A2000F0B54746CE4680B587B000920193F92372
:106A30004F00814688467F089B059F4263DA04F039
:106A40000BFE002800D1DAE04A464346484641465C
:106A500003F0E6FF04000D006A4A6B4B03F0E0FF11
:106A60006A4A6B4B03F09EF822002B0003F0D8FF1C
:106A7000684A694B04F040FA22002B0003F0D0FF73
:106A8000664A674B03F08EF822002B0003F0C8FF24
:106A9000644A654B04F030FA22002B0003F0C0FF7B
:106AA000624A634B03F07EF822002B0003F0B8FF2C
:106AB000029003910022200029005E4B03F0B0FFFA
:106AC000029A039B06000F002000290003F0A8FF94
:106AD000009A019B04000D004846414603F0A0FFC8
:106AE00002000B002000290004F006FA02000B004F
:106AF0003000390004F000FA02000B0000204E497B
:106B000004F0FAF970E002000B0003F089FF0400C2
:106B10000D003C4A3C4B03F083FF3C4A3C4B03F0E6
:106B200041F822002B0003F07BFF3A4A3A4B04F075
:106B3000E3F922002B0003F073FF384A384B03F0CF
:106B400031F822002B0003F06BFF364A364B04F07D
:106B5000D3F922002B0003F063FF344A344B03F0D7
:106B600021F82B00220003F05BFF344B02900391CD
:106B70009F429FDD324B00229F423ADC3149002088
:106B80007B182D4916001F0004F0B6F904900591FA
:106B9000002220002900274B03F042FF32003B0077
:106BA00004F0AAF9029A039B06000F0020002900B6
:106BB00003F036FF009A019B04000D004846414651
:106BC00003F02EFF02000B002000290004F094F9CE
:106BD00002000B003000390004F08EF902000B00B7
:106BE0000498059904F088F907B0C0BCB946B046CE
:106BF000F0BD154B002604920593144FC8E7002002
:106C00000D49F1E7D43888BEE9FAA8BDC4B1B4BDD6
:106C10009EEE213EAD529C804F7E923E9015CB1948
:106C2000A001FA3E7751C1166CC1563F4C555555DF
:106C30005555A53F0000E03F0000F03F3233D33F01
:106C40000000E93F0000E0FF0000E73F0000D23F06
:106C5000F0B5DE4657464E464546E0B5DD4CA54408
:106C60000D9119001400A49A0A93DB4B9200D2589C
:106C70000B00013B0493230006900892143300DAC2
:106C8000A1E31821E01E02F07FFA030001339A000D
:106C90009B1A0590DB00E318059A0793049BD41A0E
:106CA000089AD61814D40136A59F22AD361907E0EC
:106CB000A300F85804F006FD013403C5B44207D020
:106CC000002CF5DA00200021013403C5B442F7D1CD
:106CD000089B002B01DA00F0FDFB0A9922AA8C46E2
:106CE0009346089A72AB62440392069A994690467C
:106CF0000093049B9A46DB009B4408339844049B12
:106D000000240025002B13DB5F4600240025069E8F
:106D10003A687B6803CE03F083FE02000B0020007C
:106D2000290002F03FFF083F04000D004645EFD167
:106D30004B4630C3994608239C46073BE3449C4698
:106D4000039BE2449A45DAD10EA8042284465242BB
:106D50006244944608998B009C4462468446083BF2
:106D600063440B93059B0C92A59A980094460300EC
:106D7000634405930A9B8846DA00069B083B9B46C2
:106D80009344DA464346DB001900009A8C46099387
:106D9000130063441E685F684346002B32DD914652
:106DA0008E4B4344DB0099440EAB9B4600228C4B38
:106DB0003000390003F034FE04F04EFC04F082FC95
:106DC0000022884B04000D0003F02AFE02000B0095
:106DD0003000390004F090F804F03EFC5B4601C33B
:106DE0009B464B4620001A685B68290002F0DAFED9
:106DF0000822524294464B46009A06000F00E14496
:106E00009A42D3D1079B30001A0039009B4600F00C
:106E100015FDFF2300229B0504000D0003F000FE7A
:106E200000F06AFC0022704B03F0FAFD02000B0038
:106E30002000290004F060F804000D0004F00CFCB0
:106E4000814604F03FFC02000B002000290004F002
:106E500053F85C4606000F00002C00DC85E043463A
:106E6000591E89000EAB5B5818201A00001B024106
:106E7000914482409D1A0EAB5D5017231B1B1D4190
:106E8000002D00DD7EE0002200233000390002F0FA
:106E900077FA002800D1E9E04346591E089B8B424F
:106EA0000FDC0EAA94460022504B0C9843449B00E2
:106EB00063441C68043B22438342FAD1002A00D079
:106EC00023E1089B0EAA013B9B00D358002B00D066
:106ED00016E10B9A01331168043A01330029FAD004
:106EE000012242449346434403930A9B22AA43440B
:106EF0009046009ADB0094469844099B6344994667
:106F00005B46059A9B00D05804F0DCFB43461860B2
:106F10005960049B002B25DB474600240025069E74
:106F200002E00836386879683268736803F078FDE3
:106F300002000B002000290002F034FE083F04008C
:106F40000D005645EDD14B469C60DD6001239C460B
:106F50000733E3449C46039BE044E1449B45CFDD7B
:106F600098460FE700240025EDE7079B002B00D093
:106F7000BDE04346013B9B000EAAD558ED15002D00
:106F800000DC80E701239C464346E144002B00DC03
:106F90002FE20E9C002C00D09FE04346012B2FD007
:106FA000012241460FAB1C68002C00D198E08846B6
:106FB000531C802149049200091B0EA8815098455A
:106FC0001DDD414684469B008900C2586144084843
:106FD000634410E094FDFFFFA8C70000FFFFFF1F00
:106FE0000000703E0000704100002040FFFFFF3FA6
:106FF000FFFFFF001A68821A04C38B42FAD10124F2
:10700000079B002B0EDD012B00D1D1E1022B09D112
:1070100043465A1E92000EAB9B580EA903939B0247
:107020009B0A8B50022D00D02DE732003B00002040
:10703000934903F061FF06000F00002C00D122E706
:10704000079A00208E4900F0F9FB02000B00300087
:10705000390003F051FF06000F000022002330002A
:10706000390002F08DF9002800D015E74B46069351
:10707000079B30005A423900049500F0DFFB0022E4
:10708000804B04000D0002F09FF9002800D1EEE1D2
:107090007D4B00222000290003F0C2FC04F0DCFA42
:1070A00042460600970004F00DFB0022754B03F0EA
:1070B000B7FC02000B002000290003F01DFF04F0C4
:1070C000CBFA0EAAD0514246079B013218330392E5
:1070D000079393000EAAD65032E00123002268E7FE
:1070E000013204338A4200D05DE7884688E70022F7
:1070F000664B02F069F9002800D069E10025C2E67C
:10710000012343449B460393EFE64B460A00069354
:10711000079B0391183B190007930EA89300C358CF
:107120000495002B0CD18446594B43449B00634487
:107130001868043B013A18390028F9D003920791E6
:107140000020079A4E4900F079FB039B04000D00D4
:10715000002B00DAC1E10EAA9446D9009E00009BE4
:1071600066441A008C46624417009346984605917F
:10717000306804F0A7FA22002B0003F051FC424BC8
:107180003860796000222000290003F049FC043EA9
:107190003B0004000D00083F9845E9D100239946C3
:1071A0004AAB0093089B9A46534600240025002BC7
:1071B00021DB8020374B5F469846002400250026BF
:1071C0003549C00508E008239C460837E044B1452E
:1071D00011DB4346186859683A687B6803F020FC65
:1071E00002000B002000290002F0DCFC0136040044
:1071F0000D00B245E7DA009A4B4694460822DB00C0
:107200006344524294461C605D604B46039A0133CE
:10721000E344914501D09946C6E7009B9A46A49B5A
:10722000022B3BDC002B00DDE5E01CD10025002417
:107230005746059E5644326873682800210002F0C4
:10724000B1FC330005000C00083E9F42F3D1049BC3
:10725000002B03D080231B069C4664442A00230095
:107260000D990A604B600720069B18409B239B00EA
:107270009D44F0BCBB46B246A946A046F0BDC04600
:107280000000F03F000070410000703E0000E03F51
:10729000FEFFFF3F68C70000FB21F93FA49B032BC3
:1072A000E1D1039B002B00D12DE1984A059B944628
:1072B00053441C685D68039B63449B46DB00534456
:1072C0009846434620001E685F68290032003B0054
:1072D0000094019502F066FC02000B0004000D0012
:1072E0003000390003F008FE009A019B02F05AFCBE
:1072F00043469860D9601C605D6008235B42C146CC
:107300009C46E044CA45DCD1039B012B00DCFAE03B
:107310005B46DB009946D046059EC8445644346817
:107320007568434620001E685F68290032003B00F4
:107330000094019502F036FC02000B0004000D00E1
:107340003000390003F0D8FD009A019B02F02AFCBE
:1073500043469860D9601C605D6008235B424646E6
:107360009846B044C245DCD14C460027002508347D
:107370005444380022686368290002F013FC083C7A
:1073800007000D00A642F4D1049B002B7AD14A9B42
:107390004B9C0D993A000B604C605346DC689B682F
:1073A000009301948B60CC602B000A614B615AE71B
:1073B00043465A1E92000EAB9B580EA903935B02E4
:1073C0005B0A8B502EE6182300225B42059262E492
:1073D00001239C4643460225E144002B00DDD8E50D
:1073E00032003B0000204A4903F086FD06000F00F2
:1073F00049E5002404E6002500245746059E56442E
:10740000326873682800210002F0CCFB33000500CD
:107410000C00083E9F42F3D1049B002B48D123006F
:107420002A000D990A604B604A984B9903F064FD5D
:10743000039B07000E00002B13DD01244CAD380028
:107440000CCD310002F0AEFB039B013407000E00AF
:10745000A342F4DA049B002B03D080231B069C4636
:1074600066443A0033000D998A60CB60FBE64346E0
:10747000200029009E0004F0EFF80EAB985143461F
:1074800003935DE6802051460006844649680D98C6
:1074900061440B004A9A6446026043605346D968CF
:1074A0009A6865440B198260C36007614561DAE63A
:1074B00080234A984B990D9A1B06E3185360156078
:1074C00023002A0003F018FD039B07000E00002B89
:1074D000B3DCC2E772AB009336E4A49B022B06DC5C
:1074E000002B0DDC00D0BEE600250024AFE6A49BF7
:1074F000032B00D0B7E64AAB002700259A4643E7A6
:107500000025002488E700273D003DE7FFFFFF1F1F
:107510000000F03FF0B5CE46474680B587B00092F8
:107520000193F9224B00814688465B0892059342FD
:1075300007DA4846414604F08FF84A464346002899
:107540004AD04A4643464846414603F069FA040099
:107550000D0002000B004846414603F061FA3B4A29
:107560003B4B06000F002000290003F059FA394A6E
:10757000394B03F0C1FC22002B0003F051FA374ACB
:10758000374B02F00FFB22002B0003F049FA354A7B
:10759000354B03F0B1FC22002B0003F041FA334BD2
:1075A000334A02F0FFFA0E9B02900391002B1AD18E
:1075B00002000B002000290003F032FA2D4A2E4B66
:1075C00003F09AFC32003B0003F02AFA4A46434695
:1075D00002F0E8FA02000B001000190007B0C0BC6E
:1075E000B946B046F0BD002200980199234B03F044
:1075F00017FA029A039B049005913000390003F0BA
:107600000FFA02000B000498059903F075FC2200A4
:107610002B0003F005FA009A019B03F06DFC154A5C
:1076200004000D00144B3000390003F0F9F902009A
:107630000B002000290002F0B5FA02000B004846BA
:10764000414603F059FC02000B00C5E77CD5CF5A38
:107650003AD9E53DEB9C2B8AE6E55A3E7DFEB157D3
:10766000E31DC73ED561C119A0012A3F1111813F19
:10767000A6F81011495555555555C53F0000E03F36
:1076800070B50D001600040004F0CAF92900066068
:10769000200070BDD0B51900140082B000280ED0B3
:1076A000802000061B1800920193009A019B200085
:1076B00003F0B6F92222FFF7E3FF02B0D0BD2200AB
:1076C0000B00F0E7802310B500225B05FFF7E2FF17
:1076D00010BDC046E02310B50022DB05FFF7DAFF3E
:1076E00010BDC046034B48009C4640086044C00F94
:1076F0007047C04600001080474AF0B546469046A5
:107700004B005B0D98444F46D6464246C0B5050037
:107710000C000E000700132A39DC002A26DB3F4B41
:107720008446134199460B408A46034317D03C4A8E
:107730003C4B2800210002F035FA0022002301F022
:1077400039FE002809D0002C04DA8026434676034F
:107750001E4136194B4600279E43BC46B246514651
:107760006046E0BCBA46B146A846F0BD2C4A2D4B57
:107770002800210002F016FA0022002301F01AFE70
:107780000028EAD0002C2FDB00270026E5E7332A6B
:107790000EDD802384468A46DB009845DFD1020057
:1077A0000B002800210002F0FDF984468A46D6E746
:1077B0001D4A8A469446012263445242DA40844676
:1077C00091460242CBD0164A164B2800210002F007
:1077D000E9F90022002301F0EDFD0028BDD0002CC6
:1077E00009DB4B469F43B8E7640064080027254344
:1077F000B3D00E4EB1E74346142B09D03422D21A2F
:10780000012393405D19BD4204D22F00661CE8E7B6
:10781000661CE6E72F00E4E701FCFFFFFFFF0F0017
:107820009C7500883CE4377EEDFBFFFF0000F0BF55
:10783000002001497047C0460000F87F4B0070B53A
:107840005B0D14000A00002B25D14B005B0803439D
:1078500020D02B4B002203F0E3F82A4B9C4247DB5D
:107860000A004B005B0D363B274DE318AB421ADC98
:10787000002B37DC1D00353529DA244B9C4212DC05
:10788000234C244D002938DB20002900204A214BBD
:1078900003F0C6F870BD204DAB42E5D102000B00ED
:1078A00002F080F9F6E71D4C1D4D002906DB200093
:1078B00029001A4A1A4B03F0B3F8EBE7174C194D9D
:1078C00020002900154A164B03F0AAF8E2E7164CEF
:1078D000363322401B05134319000022134B03F0DB
:1078E0009FF8D7E7104C1B0522401A431100D1E73F
:1078F000074A084B03F094F8CCE7054C0C4DC3E75E
:1079000000005043B03CFFFFFE07000050C30000E2
:1079100059F3F8C21F6EA501FF0700009C7500888F
:107920003CE4377E3CE437FEFFFF0F800000903CD4
:107930001F6EA5810122F8B508210600100000F095
:10794000F1FC0724082700223900012000F0EAFC9E
:10795000320001252241022100202A4000F0E2FCF1
:107960002A003900280000F0DDFC013CEBD2F8BD14
:10797000002210B504001100022000F0D3FC20000A
:10798000FFF7D8FF10BDF7B50123002504000093D1
:10799000019572B650277F426A46AB00D058260048
:1079A0003843C0B2FFF7E4FF0020FFF7E1FF1020EB
:1079B000FFF7DEFFE020FFF7DBFF012200210220BE
:1079C00000F0B0FC3078FFF7B5FF230001368433B8
:1079D0009E42F2D1012D01D162B6F7BD34000125DE
:1079E000DAE710B5AC20FFF7C3FFAE20FFF7C0FF0A
:1079F000A520FFF7BDFF10BD70B50D0004000122EA
:107A000000F044FC29000122200000F08BFC70BD36
:107A100010B50400F820FFF7ABFF2000FFF7A8FF28
:107A200010BD10B504008120FFF7A2FF3F202040C9
:107A3000FFF79EFF10BD0000202010B5064B1B78FD
:107A40001843FFF795FF0A2000F040FE034B18781B
:107A5000FFF7E7FF10BDC0469D010010C81A0010D7
:107A6000842210B500210248520001F0C0F810BD78
:107A7000C019001010B50248FFF785FF10BDC046C1
:107A8000C019001010B508210120FFF7B5FF022131
:107A90000020FFF7B1FF00210220FFF7ADFF062114
:107AA0000220FFF7A9FF03210800FFF7A5FF03212C
:107AB0000022080000F036FC00220621022000F01F
:107AC00031FC01220621022000F02CFCFFF7C8FF48
:107AD000FFF7D0FFA220FFF74BFFA020FFF748FFE2
:107AE000C020FFF745FF0020FFF792FF0A2000F0BB
:107AF000EDFD4020FFF73CFF2C20FFF739FF32203F
:107B000000F0E4FD2E20FFF733FF322000F0DEFD11
:107B10002F20FFF72DFF0A2000F0D8FDFFF78CFF84
:107B2000AF20FFF725FFA420FFF722FF10BD0000C4
:107B300070B505000024054B2900E05C044B0134BE
:107B4000C01800F011FC0A2CF5D170BDB8C70000B8
:107B500000400440F7B50E4E3468002C16D11020BA
:107B6000FFF7E6FF0B4D2B786F78180000223900E5
:107B70000193013400F08AFB01223900019800F0E2
:107B8000D1FB02350A2CEED101233360F7BDC0468C
:107B9000CC1A0010C2C70000F8B500250B4C26789F
:107BA000677801223900300000F070FB01350022B7
:107BB0003900300000F0B6FB02340A2DEFD100206E
:107BC000FFF7B6FF0022024B1A60F8BDC2C70000E3
:107BD000CC1A001070B50500FFF7BCFF002D09D0CE
:107BE00001220721022000F051FB00220721022080
:107BF00000F098FB0B21002000F06AFB0124002814
:107C000005D00B21002000F063FB44424441002DCD
:107C100009D000220721022000F038FB01220721B1
:107C2000022000F07FFB200070BD012210B5100083
:107C30000B2100F02BFB00220B21012000F072FB36
:107C400001220221032000F021FB00220221032057
:107C500000F068FB10BD000037B51021224A050076
:107C6000136801208B4313608023204A9B01116815
:107C70001F4C0B4313600B21002200F007FB002276
:107C80000B21012000F04EFB9F211A4B1A688A43FA
:107C90001A601A6818491A60184B186801F074FACB
:107CA0000302802018432A0002212060032000F0F4
:107CB00039FB142000F00AFDFF2223689343236060
:107CC00022680F4B13430F4A236013680193019BF3
:107CD000002BFADA23680C4A13402360FFF7A5FF54
:107CE00001980004800D3EBD38820440808004402D
:107CF00000C001409840044000093D00E01A001017
:107D0000800000012CC00140FFFFFFF810B50D4CB2
:107D10002068002814DA00202060FFF79DFF0A2861
:107D20000BDC0120FFF798FFC0230138FF385B0010
:107D3000984202D8803BFF3B2360FFF776FF206824
:107D400010BDC046A001001010B5FFF7DFFF0028EE
:107D500001D1002010BD0120FFF77EFF011EF8D0E9
:107D6000014801F011FAF5E750BB12000222074B5F
:107D700010B51A60064BA0321960064B1A7001321A
:107D800058709A7001F010F910BDC046CC1C00105C
:107D9000B81C0010A41C00100022064B023110B5C4
:107DA0001960054B1A60054BA2321A70587001F029
:107DB000FBF810BDCC1C0010B81C0010A41C001057
:107DC00070B505000E00032431002800FFF7CEFF38
:107DD0000223FF33984202D0013C002CF4D170BD45
:107DE00070B505000E00032431002800FFF7D4FF12
:107DF0000223FF33984202D0013C002CF4D170BD25
:107E00000A4B10B51B68002B0ED0094CA31CA270A6
:107E1000140A5C70140C120EDA709C70FFF7E0FF0D
:107E2000831EFF3B5A425341180010BDD01A001068
:107E3000A41C001070B50E4C2468002C15D00D4CFD
:107E4000160AA270E670160C120E6271A371A21DC2
:107E500026711C0A54701C0C1B0E9470D370FFF713
:107E6000BFFF841EFF3C63425C41200070BDC046E2
:107E7000D01A0010A41C0010064B10B5186800287A
:107E800007D007210220FFF79BFF0238FF3843424B
:107E9000584110BDD01A0010064B10B518680028C4
:107EA00007D007210220FFF79BFF0238FF3843422B
:107EB000584110BDD01A0010012110B50800FFF77D
:107EC0007FFF0223FF3398420FD10120084B186037
:107ED000084B1C78230706D00323074A23400100E0
:107EE0009370FFF77DFF200010BD01246442FAE784
:107EF000D01A0010BC1C0010A41C001010B5FFF715
:107F0000DBFF01210220FFF75BFF0223FF339842D2
:107F10000FD1084B1B787F2B06D984220721022022
:107F2000054B5204FFF786FF04210920034AFFF79F
:107F300067FF10BDBC1C001002011400808080800F
:107F40000A23021153430F2210401818704770B5CE
:107F50000A21050001F018F90A210401280001F0A6
:107F6000F9F92000084370BDC12210B5520002216A
:107F70000E20FFF745FF0122014B5A7110BDC0468C
:107F8000D61A001010B5084C6379002B01D1FFF709
:107F9000EBFFA2792379520001211A430C23080038
:107FA0001A43FFF72DFF10BDD61A001010B5054B70
:107FB0001A79002A05D000221A711A72DA70FFF7B6
:107FC000E1FF10BDD61A001070B51D4C0D00617890
:107FD0002378A27809021943E378120411431B069F
:107FE000184A0B4313401A0A237062701A0C1B0EB6
:107FF000E37063792179A2701B02134A0B4313408B
:1080000023711B0A06006371A079FFF799FF0F4BDC
:108010001B881B1833806079FFF792FFB070E078FF
:10802000FFF78EFFF070A078FFF78AFF2870607866
:10803000FFF786FF68702078FFF782FFA87070BD99
:10804000BC1C00107F7F3F3F071F0000D41A0010A8
:10805000F7B504880E00050064212000019201F0AC
:108060008FF8114B8FB2E41B1C80B078FFF76FFFC5
:108070000E4CA0707078FFF76AFFE0703078FFF761
:1080800066FF2071E878FFF762FF019B6071A371C2
:10809000A878FFF75CFFE0713800FFF758FF207207
:1080A000FFF7FAFEFEBDC046D41A0010A41C001053
:1080B00070B5962283780688050000205201B61814
:1080C000010002229A424141761A022B00D80C305C
:1080D000C0189923033858436E240521023001F05B
:1080E00053F86421FF3474430419B0102418494232
:1080F000300001F049F8C82124184900300001F08F
:1081000043F8034B2018EC78C018001970BDC04626
:10811000D382FFFF10B5002848D08021254A13687C
:108120008B431360012324490A681A42FCD00322BE
:10813000224B1A6001230021214A13601160136051
:1081400011681942FCD01F4A1F49136080230C6834
:108150005B0223430B60002804D1802315490C687F
:1081600023430B60194B196881421ED01860431ECF
:108170009841174B40421840164B1168C01800F048
:1081800079FFFA21144B89001860040000F0FCFF0D
:108190001E23C8214343114A20001360490100F007
:1081A000F3FF0F4B186000F069FD10BD034B186022
:1081B000C0E7C046388204400C8004407080044010
:1081C000748004407880044080800440A401001042
:1081D00000512502001BB700E01A0010E81A001039
:1081E000E41A001010B500F043F8134A0021136898
:1081F0001B0B1B031360114A13681B0B1B0313603B
:108200000F4A13681B0B1B0313600E4A13681B0BEA
:108210001B03136001220C4B19600C4B1A60196090
:108220001A6019681142FCD02322094B01201A6000
:10823000FFF770FF10BDC046008000500080015065
:10824000008002500080035040800440448004407D
:108250000880044010B5034B034A04481A6000F03C
:108260009AFC10BDEC1B0010EC1A0010E4C70000D3
:108270004023044A11680B4313600122024B1A7019
:108280007047C04680800440F01B00100E4B70B554
:108290001B7804000E001500002B01D1FFF7E8FF4A
:1082A000631E022B0AD8094B2004C0180123026860
:1082B000B340012D04D11343036070BD0348F5E7BB
:1082C0009A430260F9E7C046F01B0010008000509E
:1082D0000F4B70B51B7805000C00002B01D1FFF788
:1082E000C7FF0020032D0BD82800012300F0B8FEA3
:1082F00002090B0D074AA34010681840431E98411D
:1083000070BD054AF7E7054AF5E7054AF3E7C046B9
:10831000F01B0010FC3F0050FC3F0150FC3F02509E
:10832000FC3F03500E4B70B51B7804000E00150087
:10833000002B01D1FFF79CFF631E022B0AD8094BCB
:108340002004C01801230268B340012D04D1134357
:10835000036070BD0348F5E79A430260F9E7C04641
:10836000F01B0010FC3F0050084B70B51B78040058
:108370000D00002B01D1FFF77BFF182223689343E8
:10838000236021680D43256070BDC046F01B0010BE
:108390003F224021044B1A60044B3E3A1A60044AC3
:1083A00013688B431360704724800440D8800440D6
:1083B000388204404021044A10B513688B4313608F
:1083C000FFF7E6FF10BDC0463882044010B500F04C
:1083D000B1FDFFF7E1FB00210948FFF7C5FF0021D0
:1083E0000848FFF7C1FF00210748FFF7BDFF002144
:1083F0000648FFF7B9FF00210548FFF7B5FF10BD9C
:108400000840044000400440AC4004401440044094
:108410001C40044010B5012000F03CFD10BD0000E0
:108420008022114B10B5DA679218DA678022D200E9
:10843000DA6780225201DA6780221201DA6780222D
:108440009200DA6700230121084A49421360084A72
:108450001160084A1360084A13600122074B1A6032
:10846000FFF7D8FF10BDC04604E100E004820440DD
:108470000882044004C000403CC0004000C00040EE
:10848000064A10B5136801331360054B1868FFF7EF
:1084900041FEFFF7C5FFC046C04610BDF41B0010EB
:1084A000A4010010F0B585B00C00019072B6FFF782
:1084B0008DFF524B524D1A68524B1A60019B5A1E47
:1084C00093413F225B4293434F4A9B184F4A1360AC
:1084D00004234F4A11680B43136000232B60A3074A
:1084E0001AD04C4A4C4913680B40136029684B4B17
:1084F000A20700D47DE0EC2252010A432A608022C8
:108500001A6092181A608022D2001A6080225201EA
:108510001A60802212011A60019B002B53D00024A4
:108520003F4B404F404E3C601C60404B21001C6064
:108530003F4B30001C60FFF717FF2200092120008D
:10854000FFF7A4FE220009212000FFF7EBFE8021A7
:10855000384A394813680B43136007223368763969
:10856000934333603368053A13433360019B5843A8
:1085700000F080FD0322314B31491860314B1C6003
:10858000314B1A60314B1A680A4080211A601A6810
:108590000A431A608023214A1E499B0013600A681F
:1085A0001A430A602A68022113432B600123284AD8
:1085B0001360284A1160284A136014601360116820
:1085C0001942FCD03B600122244B52421A60244BDA
:1085D0001A68039262B630BFC046039A1B689A427B
:1085E00005D1204B1868FFF795FDFFF719FF05B07F
:1085F000F0BD802212010A432A608AE738820440D3
:108600000482044034820440FF1800003082044099
:1086100010ED00E0008204407FE2FFFF00E100E097
:108620000400014004C00040644004400440014094
:108630000480014080800440841E000018C0004077
:108640000FF0FFFF08C0004014C000403CC00040D5
:1086500078800440708004407480044008820440A4
:10866000F41B0010A401001010B5FFF71BFF10BD94
:10867000074B1A68013203D106490A6801320A60C1
:108680001A6801321A60044A136801331360704794
:10869000001C0010FC1B0010F81B001080235B0462
:1086A00098420AD20023054A01381360044A106038
:1086B000044A13600722044B1A607047001C001024
:1086C00014E000E018E000E010E000E00B4A13685E
:1086D000002800D10130C143994209D2591C081821
:1086E0001168994200D2704711688842FCD8F7E7B8
:1086F0001168C91A8142FBD3F5E7C046001C00107F
:10870000014B18687047C046001C00100122034B43
:108710001A60034A136801331360704700C00040B9
:10872000041C00100122034B1A60034A1368013332
:108730001360704700000140081C00100122034B29
:108740001A60034A13680133136070470040014008
:108750000C1C00100122034B1A60034A13680133FA
:108760001360704700800140101C00100E22174B50
:1087700010B51B681340062B12D1154B90321B68A5
:10878000134205D0134ADBB25360134B1B6810BD74
:10879000DB07FCD5104B1868C0B200F0A7F8F6E76D
:1087A000042BF7D00C2B05D10A4AF43351680B4344
:1087B0005360ECE7022BEAD1054B1A68054B920691
:1087C00002D500229A60E2E70122FBE70880004020
:1087D00014800040141C00100080004000487047C6
:1087E000141C0010F7B58022002107252A4B2B4CC2
:1087F0009203070001912000DA67902200F0F7F958
:10880000019B274EA360274B1A68AA431A600122D6
:10881000196811431960244B1968A9431960196834
:1088200011431960802321495B01086803430B60F1
:108830001F4B1A60823232601E4A126819681E4B42
:108840001868504300F016FC3900000900F012FCD3
:1088500010221A4B1A491A60030A0B600323194F9E
:10886000C0B2386060203360174B1D60174B1A6828
:1088700001921A680240602AFBD15F3A18681042E0
:1088800007D122708022124B92031A6005230B60DD
:10889000F7BD38680190F1E704E100E0141C001016
:1088A0000C800040A4400440A84004408080044064
:1088B0009880044078800440E01A0010288000402E
:1088C0000480004000800040088000401480004088
:1088D00000E100E0202303490A681A42FCD0024B61
:1088E00018607047148000400080004010B50400FC
:1088F000FFF774FF437BC318DC73437B0133DBB2A8
:1089000043735BB2002B01DA0023437310BD70B5D3
:1089100004001D0000202E5C2318002E09D1121A1D
:10892000D518EC1A002C07DCD343DB171A401018BB
:1089300070BD26540130EEE719700133F1E7F8B548
:10894000541E0F001E00050023000100092E16D939
:108950000A21300000F08EFB2200030039002800BD
:10896000FFF7EDFF04002D1830000A2100F008FC8D
:1089700030312970601CF8BD0F70013B0131002BB4
:10898000FADC0020824200DD20002D18002A00DCE5
:108990000122541EE8E7F7B50E00D9175F1804004E
:1089A00001934F40551E092F17D90A21380000F0B6
:1089B00061FB019A0300002A00DA43422A002000EA
:1089C0003100FFF7E8FF0500241838000A2100F005
:1089D000D7FB3031681C2170FEBD019B002B00DAF3
:1089E000951E23006119CA1A002A0CDCE843019A7B
:1089F000C017054064196B1C002AE6DA2D221D0001
:108A000022700134E1E71E700133ECE7F7B51E0078
:108A1000089B1400013A1F0905001300002F11D014
:108A200033000097FFF7F2FF2D180F23089F1F4018
:108A3000FAB2092F12D830322A700130FEBD01700F
:108A4000013B0130002BFADC0020844200DD1000E5
:108A50002D18201E00DC01200138E6E7002E01D091
:108A60003732E9E75732E7E7F0B505000F001C00A1
:108A700085B0002801D00023037000261378002B56
:108A800000D16DE0B74204D80023013D2B70013EB8
:108A900032E0252B04D001322B7001360135EDE791
:108AA0005178252902D129700232F6E7931C0393ED
:108AB000302902D02021531C0393039B1B782D3BAC
:108AC0005A425341039AD31800220393039B1B7805
:108AD00018003038092812D99019B84201D9BA1BA8
:108AE000D2B2692B1FD013D8632B35D0642B1AD088
:108AF000582B2DD001267642300005B0F0BD0A205B
:108B000042439A18039B303A0133D2B20393DDE714
:108B1000752B11D0782B14D0732BEBD1280008CCF7
:108B2000FFF7F5FE03E0280008CCFFF734FF039AB7
:108B30002D1801323618A1E7280008CCFFF7FFFEF8
:108B4000F5E708CC009300232800FFF75FFFEEE76E
:108B500008CC00930123F7E708CC01202B70E6E74F
:108B6000B74200D890E72B70C6E710B513000A0093
:108B70006421FFF779FF10BD00B59BB00A0001002A
:108B800001A8FFF7F2FF632800DDFEE701A800F06F
:108B90009BF81BB000BD0FB407B504A901C9019132
:108BA000FFF7EAFF03B008BC04B0184770B5060031
:108BB0000E430325340003002C402E420FD1AA425D
:108BC0000DD90B5903510434131B032BF9D803247B
:108BD000131F9B0801339B00C9182240C3180024AF
:108BE000A24200D170BD0D5D1D550134F8E770B58E
:108BF000830704D003009A189A4217D170BD03006E
:108C0000032AF8D90C040B0623430B430C0223431D
:108C10000400861808C4351B032DFBD80324131F3A
:108C20009B0801339B00C3182240E4E7197001330D
:108C3000E2E710B5814208D20139431E002A00D173
:108C400010BD8C5C9C54013AF8E78142F8D90023AE
:108C500002E0CC5CC45401339A42FAD1F0E703003D
:108C600000201A5C002A00D170470130F9E7002388
:108C7000CA5CC2540133002AFAD17047FA21094B69
:108C800010B51868890000F07FFAFFF707FD9620FD
:108C90000002FFF7A7FD012000F0FCF8FFF72EF916
:108CA00010BDC046E01A001010B5FFF79BFAFFF7A1
:108CB000DFFAFFF77FFBFEF7E5FEFEF7D1FEFFF7D9
:108CC000C9FAFFF7DBFF10BD10B5040020780028BB
:108CD00000D110BD0134FFF7FDFDF7E78022102120
:108CE0000820064BD2051160186080235B011068D4
:108CF000084202D0013B002BF9D170471800004018
:108D0000594A10B5136801331360584B584A1B6811
:108D1000DBB2302B00D176E018D8182B5AD005D80A
:108D2000082B37D0102B46D0082351E0202B00D140
:108D30007AE0282BF8D14F4B4F49186809688842D0
:108D400052D21968481C18604C4B48E0482B00D19F
:108D50006AE00AD8382B60D0402BE5D1484B19681F
:108D6000042301295DD11360DEE7502B66D0582B18
:108D7000DAD14448444B1B680168DBB24C1C0460E8
:108D8000424843540221424BFF3119608023F1399C
:108D9000DB0530E00021374B19601968481C18606A
:108DA000364B5B5C3849DBB20B6028231360012231
:108DB000374B1A6010BD0021324B19602D490B68EA
:108DC000581C08602D49CB5C2F49DBB20B6028236F
:108DD0001360EFE727490B68581C086027495B5C64
:108DE0002949DBB20B609FE7254B19688023DB051F
:108DF000002902D02021196096E702202449FF3083
:108E000008601021F7E780231021DB051960082393
:108E1000136081221E4B5200CBE782211C4B49007C
:108E2000E9E78021C905DDE780231021DB05196012
:108E3000082313600422164BFF32BAE71149124B84
:108E40001B680868DBB2441C0C60104C23540C4BAC
:108E50001B680868013B0421834202D98023DB059B
:108E6000C9E7116060E7C046D81C0010040000404C
:108E700018000040D41C0010CC1C0010A41C0010D2
:108E8000B81C0010D01C001008000040BC1C0010D2
:108E9000B41C001002231B4A70B511681A4D0B4315
:108EA00013602023194A040011680B431360184B08
:108EB0001A682A401A600122186810431860154B7E
:108EC00019682940196019680A431A606C22124B0C
:108ED00012491A60124B186800F056F9114B1860CD
:108EE000114B1860022C02D1A022104B1A60802274
:108EF0000F4B12021A6080234022DB0501201A600A
:108F000070BDC04604800440F8FCFFFF8080044030
:108F1000304004403440044018000040400D03003D
:108F2000E01A001014000040100000400C00004047
:108F300000E100E08022164B120210B5DA676C22C5
:108F4000144B15481A60154B1968014019601A68CE
:108F500004211A60124B1A6802401A601A68002035
:108F60001A600122FFF792F9012204210020FFF785
:108F7000D9F9012205210020FFF788F901220521F6
:108F80000020FFF7CFF90022064B1A6010BDC04643
:108F900004E100E018000040F8FCFFFF304004400E
:108FA0003440044004800440F8B50023164A174CAE
:108FB000202123601360164A13608022D2051160BD
:108FC000144A2168012907D0934203D1FFF786FE96
:108FD0000020F8BD0133F4E79342F7D000250E4F8F
:108FE0003E68013E2368FF2B01D92068F1E73B680A
:108FF000B34204D03E68FFF783FB0A300500FFF759
:109000007FFBA842EED1E1E7D01C0010B41C001099
:10901000D41C0010FF0F0000D81C0010FEE7FEE774
:1090200010B50A4A0A4B0B498B4207D300210A4B61
:109030000A4A934207D3FAF7BDFAFEE710780132E5
:1090400018700133F0E719700133F2E7F8C8000037
:1090500000000010D8050010D8050010DC1C00101E
:1090600002B4714649084900095C49008E4402BCBB
:109070007047C046002243088B4274D303098B42D9
:109080005FD3030A8B4244D3030B8B4228D3030CD8
:109090008B420DD3FF22090212BA030C8B4202D37A
:1090A0001212090265D0030B8B4219D300E0090AA2
:1090B000C30B8B4201D3CB03C01A5241830B8B42AB
:1090C00001D38B03C01A5241430B8B4201D34B0394
:1090D000C01A5241030B8B4201D30B03C01A5241F9
:1090E000C30A8B4201D3CB02C01A5241830A8B427E
:1090F00001D38B02C01A5241430A8B4201D34B0267
:10910000C01A5241030A8B4201D30B02C01A5241CA
:10911000CDD2C3098B4201D3CB01C01A524183097E
:109120008B4201D38B01C01A524143098B4201D3B8
:109130004B01C01A524103098B4201D30B01C01AE3
:109140005241C3088B4201D3CB00C01A524183085D
:109150008B4201D38B00C01A524143088B4201D38A
:109160004B00C01A5241411A00D2014652411046EA
:109170007047FFE701B5002000F0F0F802BDC046DF
:109180000029F7D076E7704703460B437FD40022CF
:1091900043088B4274D303098B425FD3030A8B428B
:1091A00044D3030B8B4228D3030C8B420DD3FF22F5
:1091B000090212BA030C8B4202D31212090265D0C3
:1091C000030B8B4219D300E0090AC30B8B4201D376
:1091D000CB03C01A5241830B8B4201D38B03C01ABD
:1091E0005241430B8B4201D34B03C01A5241030B34
:1091F0008B4201D30B03C01A5241C30A8B4201D3E5
:10920000CB02C01A5241830A8B4201D38B02C01A8F
:109210005241430A8B4201D34B02C01A5241030A06
:109220008B4201D30B02C01A5241CDD2C3098B42EB
:1092300001D3CB01C01A524183098B4201D38B0168
:10924000C01A524143098B4201D34B01C01A52410B
:1092500003098B4201D30B01C01A5241C3088B4250
:1092600001D3CB00C01A524183088B4201D38B003B
:10927000C01A524143088B4201D34B00C01A5241DD
:10928000411A00D201465241104670475DE0CA0FB4
:1092900000D04942031000D34042534000229C4674
:1092A00003098B422DD3030A8B4212D3FC2289017E
:1092B00012BA030A8B420CD3890192118B4208D354
:1092C000890192118B4204D389013AD0921100E0B6
:1092D0008909C3098B4201D3CB01C01A52418309CA
:1092E0008B4201D38B01C01A524143098B4201D3F7
:1092F0004B01C01A524103098B4201D30B01C01A22
:109300005241C3088B4201D3CB00C01A524183089B
:109310008B4201D38B00C01A5241D9D243088B42F1
:1093200001D34B00C01A5241411A00D20146634694
:1093300052415B10104601D34042002B00D54942F8
:10934000704763465B1000D3404201B5002000F037
:1093500005F802BD0029F8D016E770477047C046EF
:109360008446100062468C461900634600E0C04601
:109370001FB501F0F1FA002801D40021C8421FBD39
:1093800010B501F041FA4042013010BD10B501F0B6
:10939000E3FA002801DB002010BD012010BDC0460B
:1093A00010B501F0D9FA002801DD002010BD012020
:1093B00010BDC04610B501F069FA002801DC00209C
:1093C00010BD012010BDC04610B501F05FFA0028A5
:1093D00001DA002010BD012010BDC046002B15D1C0
:1093E000002A13D1002906DB01DC002806D000206A
:1093F000C043410802E080210906002007B402486A
:1094000001A14018029003BD55FFFFFF03B4684659
:1094100001B5029800F0A4F8019B9E4602B00CBC76
:109420007047C046F0B5CE46474680B5070099461E
:109430003B0C9C4613041B0C1D000E0061460004EF
:10944000140C000C45434B4360436143C0182C0C83
:1094500020188C46834203D980235B029846C4447B
:10946000494679437243030C63442D042D0CC918FB
:10947000000440198918C0BCB946B046F0BDC046CA
:1094800070B500220C4B04000D00FFF79DFF002873
:1094900004D12000290002F0DFF870BD064B002245
:1094A0002000290001F028FD02F0D6F880231B06D9
:1094B0009C466044F1E7C0460000E04170B50500FD
:1094C0000C000022002328002100FFF75FFF002886
:1094D00008D12800210000F00FF802000B00100056
:1094E000190070BD80231B06E118280000F004F865
:1094F000002342428B41F2E770B500220B4B0D0076
:10950000040001F08DFAFFF7BBFF060002F00AF934
:109510000022074B01F084FA02000B002000290012
:1095200001F0EAFCFFF7ACFF310070BD0000F03D38
:109530000000F04170B50600080002F0C3F80022F8
:10954000064B01F06DFA0D000400300002F0EAF85D
:109550002B00220000F026FB70BDC0460000F04149
:10956000F8B5CE46474680B59146984604000D00B2
:1095700002F070F907000E0002000B004846414659
:10958000FFF750FF241A8D41089B380031001C6002
:109590005D60C0BCB946B046F8BDC046F0B5C64631
:1095A00043025B0A4E0245004F00DA00C40F9C469E
:1095B000700A904600B52D0E3F0EC90FB6098C42B9
:1095C0004BD0EA1B002A36DD002F61D0FF2D00D1E1
:1095D000ADE08023DB041E431B2A00DCD3E0012026
:1095E0004346181A430100D48CE0800187093800F3
:1095F00002F006F905388740854200DCB6E02D1AF6
:10960000B3483840430704D00F230340042B00D055
:109610000430430100D478E06A1CFE2D65D080013F
:10962000430A9C46D2B26346D0051843E407204360
:1096300080BCB846F0BD002A35D07A1B002D00D082
:10964000AFE04346002B00D1A7E0531E012A00D112
:109650002FE1FF2A69D01A00AAE0E91B002970DD7A
:10966000002F37D0FF2D62D08023DB041E431B293F
:1096700000DCB0E001204044430143D50135FF2D1B
:1096800033D00123934A0340400810401843B9E700
:10969000002E00D183E0511E012A00D1D8E0FF2A1C
:1096A00045D00A0098E7FE276A1C174200D086E0E2
:1096B000002D00D0B7E04346002B00D1F3E000229C
:1096C000002EB0D0981B430100D4FAE043460C00B2
:1096D000F01A97E7002E00D1C8E04A1E012900D1F8
:1096E000AEE0FF2923D01100C1E70023FF229C46F2
:1096F00099E7FE216A1C114277D0FF2AF5D01500A8
:1097000046447008430700D07EE7C308FF2D0ED003
:109710005B025B0A9C46EAB285E7002E07D08022F6
:10972000D203134203D0104201D10C000300002BDE
:10973000DBD08020C00318434002430A9C46FF222E
:1097400071E70029D5D07A1B002D60D14346002B4C
:1097500024D0531E012A73D0FF2AE7D01A001B2AF7
:1097600000DC85E001203D00801985E720233A00D8
:10977000451B38000135EA405D1BA840431E984157
:10978000002510433EE7202330009B1A310098400B
:10979000D140431E9841084322E70C000300150006
:1097A000B4E7FF2FC1D080234046DB041843804636
:1097B0001B2A51DD01200C003D00301A12E7434600
:1097C0009F1B7B012BD4002F00D010E70023002427
:1097D00000229C4627E7202332003000CA40591A55
:1097E0008840431E9841104345E7002D4AD1434627
:1097F000002B63D00022002E00D114E7300040443B
:10980000430100D47EE7324B013518407AE7FF2F41
:109810008CD080234146DB04194388469FE74346AA
:109820000C00F71AE3E64246002A00D075E7002E46
:1098300000D07AE78023DB0300249C46FF22F2E677
:10984000300040440125430100D45BE7022518E7BE
:1098500043460125981BC5E6202344464046D44094
:109860009A1A9040431E98412043A4E70D004DE70B
:10987000202341464046D1409A1A9040431E9841C9
:10988000084370E74246002A00D14FE7002E00D17E
:109890004DE78022D203134200D148E7104200D0A6
:1098A00045E7030043E7002E90D00C0084460022D9
:1098B000B9E643460C00F01A013593E684460022CF
:1098C000B1E6002800D01DE7002300249C46AAE64C
:1098D000FFFFFFFBFFFFFF7DF0B54F464646D64634
:1098E0004502C0B547000C1C6D0A3F0EC60F002F85
:1098F00000D170E0FF2F00D175E0EB008025ED0472
:109900001D43002399469A467F3F6002430A9846CA
:1099100063001B0EE40F002B4ED0FF2B46D04246B7
:10992000D0008022D2040243904600227F3B3100C7
:10993000FF1A4B466140C9B213430F2B00D9B5E063
:109940006E489B00C3589F46002398462600454614
:1099500092465346022B00D189E0032B00D19EE0B2
:10996000012B18D03B007F33002B69DD6A0704D040
:109970000F222A40042A00D004352A0103D5604B67
:109980001D403B008033FE2B00DD70E0AD016D0A11
:10999000D8B202E00E0000200025C0052843F607DB
:1099A0003043E0BCBA46B146A846F0BD4346002B62
:1099B0003FD10222FF3F03E04346002B2DD101227D
:1099C00031004B466140C9B213430F2B34D84D4888
:1099D0009B00C3589F46002D13D104239946033B97
:1099E00000279A4691E7002D05D108239946063BAA
:1099F000FF279A4689E70C239946093BFF279A4699
:109A000083E7280001F0FCFE7627431F9D400023DA
:109A10007F4299469A463F1A77E7404601F0F0FEAA
:109A20004246431F9A4076235B4290461B1A00220F
:109A30007DE7FF2303227AE70E00FF200025ACE735
:109A40000120C01A1B28A6DC9E372A00BD40C24058
:109A50006B1E9D4115436B0704D00F232B40042B35
:109A600000D004356B0144D50120002595E7FF2087
:109A7000002592E780250026FF20ED038DE70023D7
:109A800098468020C003054209D04346034206D1D0
:109A9000454605436D022600FF206D0A7DE78020C4
:109AA000C00305436D02FF206D0A76E742466B0155
:109AB0005001834219D21B220025013F01261C00C0
:109AC0006D005B00002C01DB984201D81B1A354366
:109AD000013A002AF3D15A1E93411D433B007F33C4
:109AE0000E00002B00DD41E7AAE71A2201251B1A10
:109AF000E4E7AD0100206D0A4FE7C046F0C7000063
:109B0000FFFFFFF730C80000F8B5002813D0C317D7
:109B1000C6185E40C40F300001F072FE9E2305009F
:109B20001B1A962B0FDC082801DD083DAE4076029B
:109B3000760AD8B202E0002400200026C005304397
:109B4000E4072043F8BD992B0CDD05223100121AE1
:109B5000D1400A00010030001B318840411E88417D
:109B600002431600052D12DC31000D4F39407207FB
:109B700009D00F203040042805D004314A0102D515
:109B80009F2339405B1B89014E0AD8B2D6E76A1F72
:109B900096403100024F39407207F4D0E9E7C046E1
:109BA000FFFFFFFBF0B54F464646D6460D000400CA
:109BB000C0B51F0011002803620F400A10437A004D
:109BC000520DE3003C039146640AFA0F4F0F6E00FA
:109BD00027439246B846760DED0FC900954200D155
:109BE00099E04C46341BA446002C00DC7CE04A463D
:109BF000002A00D1B8E0C54A964200D11CE180227B
:109C00003C0012041443A0466246382A00DD61E19C
:109C10001F2A00DDCCE164462022121B44469440FA
:109C20000F00A14664469140E7404C464A1E9141D0
:109C30003C43424621436446E240801A5C1AA342F8
:109C40009B415F42C71B3B0200D4D0E07F027F0AEA
:109C5000002F00D1FFE0380001F0D2FD01000839EB
:109C6000202322005B1A8F40DA408C401743B14218
:109C700000DAFFE0891B4B1C1F2B00DDA8E020222F
:109C80003900D21A200094409140D840621E94417D
:109C9000DF40002601430C43630709D00F23234014
:109CA000042B05D0231DA342A44164423F191C008C
:109CB0003B0200D49EE0954B01369E4200D1B7E0B6
:109CC000934AE40817407B0771057F0223433F0B4B
:109CD0004A0D12053A43ED072A4318001100E0BC73
:109CE000BA46B146A846F0BD002C4BD04C46A41B4A
:109CF000A446002E00D023E104001C4300D1AFE1B4
:109D00006246541E012A00D115E2804DAC4500D1B7
:109D1000C8E1A4461BE14A46B21A9446002A00DC78
:109D2000ACE04A46002A43D0784A964200D1AFE1DF
:109D300080223C0012041443A0466246382A67DCA5
:109D40001F2A00DC5FE14746203AD7406246202ABE
:109D500005D064464022121B4446944021434A1ECB
:109D600091410C003C4357E03A000A4300D105E121
:109D70002200013A012C00D182E1644CA4455BD061
:109D8000944641E7634C771C274200D0C4E00400AE
:109D90001C43002E00D069E1002C00D1BFE14446F5
:109DA0000C4300D0D0E14207DB081343C00829E090
:109DB0003A000A4300D170E162466446013A012C40
:109DC00000D1E0E0514CA44500D161E19446B4E7F4
:109DD0003A001F39CA401100202B03D04022D31A69
:109DE0009F403C43631E9C41002700260C436307B1
:109DF00000D053E7B446E4087B072343F808434AFE
:109E000094451DD06246070352053F0B520D60E793
:109E100044460C43621E9441E4189C429B415F42BD
:109E20003F183B02E3D5394B01369E4200D0B5E0E6
:109E30003200002700234CE74207DB081343C00829
:109E40001A00024300D1E1E180273F0307433F03AB
:109E50002E4A3F0B3DE7200001F0D2FC01001831F3
:109E60001F2900DCFCE60838844027000024B142AA
:109E700000DBFFE6264A761A17400DE7002A2FD0AE
:109E80004A46921B9446002E00D1ADE01F4A9145F0
:109E900000D10FE18022120410436246382A00DD0F
:109EA0000FE11F2A00DD80E1644620221E00121B04
:109EB0006746040093409440FE405A1E9341F84088
:109EC00034431C43804464188C42BF417F424E4659
:109ED0004744A6E742460A4311004A1E9141ADE6B7
:109EE0000C4C721C224200D0A1E002001A43002E4A
:109EF00000D0FAE0002A00D145E13A000A4300D040
:109F000046E14207DB081343C0087BE7FF07000078
:109F1000FFFF7FFFFE07000047465C1AC21BA342FB
:109F2000BF417F42B94617004A46BF1A3A0200D5E0
:109F30008DE023003B4300D08AE60020002561E746
:109F4000B44CA14500D1ADE08024240420436446F4
:109F5000382C3DDC62461F2C00DDB7E020251E00BA
:109F60002D1B0400AB40AC40D640D04042465D1EA5
:109F7000AB413443121A904623432CE04207DB08DE
:109F80001343C0083BE75C189C429B4140445B4242
:109F9000C71801263B0200D429E702269E4A63081F
:109FA0001740012214401C43FB071C437F0873E643
:109FB0004446203AD4406246202A05D067464022D3
:109FC000D21B4746974039434A1E9141214335E60B
:109FD0000343581E8341CC1AA142BF4143467F42EE
:109FE00055464E46DF1B2EE602001A4300D1BDE067
:109FF00062466446013A012C00D1E5E0854CA44557
:10A0000058D0944649E764462022121B44469440A7
:10A010000F00A14664469140E7404C464A1E9141DC
:10A020003C4342460C436146CA408018F4E6794CF2
:10A03000A24200D1FDE6591899429B4140445F423B
:10A04000C719FC07490816000C437F08CFE6CC1A55
:10A05000A142BF4143467F42181A5546C71BF7E548
:10A06000C9087B0755460B43F808C8E6002C00D00A
:10A0700081E043460B4315D1802000250003E3E631
:10A080005C1AA3429B41C71B5B420126FF1ADAE51B
:10A090004207DB081343C008D2E64207DB0813433C
:10A0A000C008ACE643464246C9085B0755460B4329
:10A0B000D008C5E6434642465B07C9080B43D008B3
:10A0C000BEE603431C00631E9C41FCE60200203CEC
:10A0D000E24014006246202A03D04025AD1AA84071
:10A0E0000343581E8341234375E7002AE2D03A0018
:10A0F0000A43CDD04207DB0813438022C008120375
:10A10000104206D0FC08144203D12000CB087A0785
:10A1100013435A0FDB005207DB08134390E6434614
:10A120000B4300D109E743464246C9085B07554641
:10A130000B43D00866E6CC1AA14289413F1A494236
:10A14000554601267F1A7EE542465C1A871AA342CD
:10A1500092415242BF1A3A023DD5CC1AA1428941DE
:10A16000434649421F1A55467F1A95E57B07C908A1
:10A170000B43F80843E64446DB080C4330D1420762
:10A180001343C0085CE67B07C9080B43F80839E6AF
:10A190005C189C429B4140445B42C7183B0200D480
:10A1A00025E61D4B01261F4021E60400203AD4403D
:10A1B0006246202A04D040226646921B9040034308
:10A1C0005A1E93411C437EE65C188C4289414044F0
:10A1D00049424718DDE623003B4300D1ADE606E6E1
:10A1E000440723438024C0082403204208D0424669
:10A1F000D608264204D155463000CB0851070B4300
:10A200005A0FDB00DB085207134319E60023014A0B
:10A210001F005EE5FF070000FFFF7FFFF0B5574618
:10A220004E464546DE46E0B5814605000C03480033
:10A2300092461F0085B0240B400DCE0F002800D1A0
:10A2400056E1D44B984200D172E16B0FE4001C43FD
:10A2500080231B0423439846CF4BED009B460023ED
:10A260009946834400933C037B005046240B5B0DCE
:10A27000FF0F002B00D11FE1C64A934200D162E1DB
:10A28000C549420F8C46E40059461443802263447A
:10A290001204CB1A14439B46C200002033007B40BB
:10A2A0009A464B460F2B27D8BC499B00CB589F465C
:10A2B000B246009B022B16D0032B00D18EE2012B5D
:10A2C00000D0D9E000230024002552461B0523437B
:10A2D000D20713432800190005B0F0BCBB46B246B4
:10A2E000A946A046F0BD00240025AA4BEDE7BA46DA
:10A2F000A04615000090DCE7444500D2C7E100D13C
:10A30000C2E101235B429C462E0040460025E34407
:10A310002302140E1C431B0C994623041F0C12022B
:10A32000494600920197FEF72BFF02007A430B0487
:10A33000310C804619438A4207D901235B429C466F
:10A340000919E0448C4200D807E2881A4946FEF712
:10A3500017FF09048C4631046646019A090C4243F2
:10A36000030031438A4204D90919013B8C4200D8C9
:10A37000EDE1881A424612041A4390464146009B7A
:10A380000E041B0C1F000293009B360C1B04190CBF
:10A390000B007343120C7E43039151437A431F0C0D
:10A3A000BC4676186644B14203D9802149028C46E6
:10A3B0006244310C8A1831041E04360C8E19904206
:10A3C00002D312D1B54210D24346591E009B9C467F
:10A3D00065441F009D429B415B421B19C01884428B
:10A3E00000D2A0E100D19BE18846AE1BB542AD4151
:10A3F000801A6D42401B844200D1D5E14946FEF7E8
:10A40000BFFE019A0B044243310C050019438A42F6
:10A4100000D96CE1881A4946FEF7B2FE019A36046B
:10A4200042430904360C03000E43B24200D953E103
:10A430000398B61A02002D041D43029F2B041B0C27
:10A440005A437B439C46290C4843130C8444634481
:10A450007943984203D98020400284466144180C15
:10A4600012041B04120C41189B188E4200D2FFE00C
:10A4700000D1FAE001231D43494A5A44002A00DC76
:10A48000AAE06B0700D03DE1ED084346DB0106D5AD
:10A490004246444B1A4090468022D2005A44424BD6
:10A4A0009A4200DD1FE743465B071D4343465205C2
:10A4B0005C02240B530D08E75246224300D17BE097
:10A4C000002C00D1FAE0200001F09AF902000B3ACA
:10A4D0001D2301009B1A52460839DA408C40144370
:10A4E00052468A40314B58449B4683440020D5E66F
:10A4F0004B462343984644D0002C00D1CEE02000A8
:10A5000001F07EF9010002000B391D235B1A494658
:10A510001000D940083884400B004D46234398462C
:10A5200085402348831A9B460023994600939AE668
:10A530004B46234398461DD108239946063B0025E8
:10A54000834600938FE65246224309D102234946AF
:10A550001943184B89469C4600240220E3449DE69B
:10A5600003234A461A43134B91469C465246032006
:10A57000E34493E60C239946093BA04683460093A7
:10A5800071E60423994600239B460133002500937E
:10A5900069E6C046FF07000001FCFFFF70C800002D
:10A5A000FF030000FFFFFFFEFE070000F3030000B3
:10A5B0000DFCFFFF01F8FFFF4946012319438946BF
:10A5C000002401206AE6002380249A4600258A4B55
:10A5D00024037AE601256D4201239B1A382B00DD06
:10A5E00070E61F2B00DCBFE01F2149428A1A41465A
:10A5F000D1400A00202B04D04146804B5B44994057
:10A600000D436B1E9D4107232A431D000024154066
:10A61000134200D1D4E00F2100231140042900D1BE
:10A62000CBE0111D9142924152429B180A0019023F
:10A6300000D4C2E001230024002546E680234146E1
:10A640001B03194208D01C4206D11C432403BA46FE
:10A650001500694B240B38E68024434624031C4331
:10A660002403B246644B240B2FE6002B00D103E7F2
:10A67000A619681EA64200D28DE08E4200D2A3E049
:10A6800000D1B3E00500F5E6AA4200D939E6434619
:10A69000DE0758086B081E43ED0739E6484601F00F
:10A6A000AFF801000200153120321C2900DC2CE734
:10A6B0004B46083883400025984632E701F0A0F861
:10A6C00003001A00153220301C2A00DC00E7544633
:10A6D000083B00229C4005E73619013BB44200D9F3
:10A6E000A6E6B24200D8A3E6831E3619A0E60919F1
:10A6F000013D8C4200D98DE68A4200D88AE6851E4B
:10A70000091987E60F232B40042B00D1BCE6052353
:10A710005B42AB429B4104355B42ED089844B4E692
:10A72000AF4200D960E6824204D800D05CE6AE4277
:10A7300000D859E602235B429C46009BE0449C46BD
:10A7400065449D429B415B421B19C0184DE68A42FD
:10A7500000D80EE6831E09190BE68A4200D8F4E5FC
:10A76000831E98460919F0E52549280059448D4073
:10A7700042468A40691E8D414146D840D940024335
:10A780002A430B00510700D151E70F211140042942
:10A7900000D046E74BE705008E4200D06AE6009AFB
:10A7A000934200D066E667E6164A5A44002A00DC67
:10A7B00010E701230025984467E65D075B021C0B48
:10A7C000D2080023154380E50098023D42008242F2
:10A7D000BF417F423C1936190092DDE78024434691
:10A7E00024031C432403044B240B6EE5009A9A4275
:10A7F000EAD30500D3E7C046FF0700003E0400008F
:10A800001E040000FF030000F0B54E464546DE463C
:10A8100057469046E0B517001A03120B0500844610
:10A8200019480E034C0091465A00DB0F9B46360B2D
:10A83000640DC90F520D844219D0824210D00120FC
:10A8400094420ED14E450CD10120C44509D1594541
:10A8500017D0002C05D130002843431E984100E05A
:10A860000120F0BCBB46B246A946A046F0BD33006D
:10A8700001202B43F5D1A242F3D14B463B43F0D10B
:10A88000E2E70020EDE7C046FF070000F0B54746CD
:10A89000CE460400180016001B031B0B2D4D4A006A
:10A8A000994680B543000F03A446B0463F0B520DB6
:10A8B000C90F5B0DC00FAA4221D0AB4213D0002AB2
:10A8C00022D13C43002B02D14D462E4322D0002CF6
:10A8D00010D0814222D00220013908400138C0BC8A
:10A8E000B946B046F0BD4D462E4329D1002AF0D1DD
:10A8F0003C43EED10028F2D101204042EFE73D0079
:10A9000025431DD19342EED0002BE2D14C46264385
:10A91000DFD1E0E70020002CE1D0DCE79A420ADC3E
:10A92000E8DB4F45D7D80ED000204F45D7D20029BD
:10A93000E2D00800D3E74342584140000138CEE757
:10A9400002204042CBE7C445C5D80020C445C6D24A
:10A95000EDE7C046FF070000F0B54746CE460400CD
:10A96000180016001B031B0B2C4D4A00994680B59E
:10A9700043000F03A446B0463F0B520DC90F5B0DB9
:10A98000C00FAA420DD0AB4210D0002A27D13C43C1
:10A99000002B11D14D462E430ED10020002C15D096
:10A9A0000EE03D00254310D1934218D14D462E4371
:10A9B0000BD1002A02D13C43002C0BD0814214D091
:10A9C000022001390840013800E00220C0BCB9462D
:10A9D000B046F0BD0028F9D101204042F6E7002B37
:10A9E000ECD14C462643E9D1EAE79A4204DD4342E2
:10A9F000584140000138E9E79A42EBDB4F45DFD888
:10AA000006D000204F45E1D20029E5D00800DDE75F
:10AA1000C445D5D80020C445D8D2F5E7FF070000CB
:10AA2000F0B557464E464546DE46E0B598460C031F
:10AA30004B000600924687B0240B5B0DCF0F002B16
:10AA400000D15CE1D94A934200D175E1420FE400A4
:10AA50001443802212041443D54AC500944663442B
:10AA60000093002399469B46434642461E03D20F5D
:10AA70005B0050469046360B5B0D00D120E1CB4A7F
:10AA8000934200D162E1CA49420F8C460099634467
:10AA9000F6008C46164380229C44120463461643FB
:10AAA000C200002000930099434601318C4649467C
:10AAB0007B4001930F2926D8BE4B890059588F46F9
:10AAC000434601933400150083465B46022B16D0A3
:10AAD000032B00D103E2012B00D0CDE000220024A3
:10AAE0000025019B12052243DB071A4328001100B1
:10AAF00007B0F0BCBB46B246A946A046F0BD002454
:10AB00000025AA4AEDE7280C2D042D0C2B00110C72
:10AB10001204120C5343984613002F0043439946E6
:10AB20004F434F44BB4647460B003F0CBA46434396
:10AB3000DA440293D14504D980277F02B9464B44B9
:10AB4000029353461B0C9B4653461F0443461B046B
:10AB50001B0C98463B0043440493330C3604360CDC
:10AB60009846330043439946434643432F009A4651
:10AB7000434677435D43380C4D444519A94503D9F5
:10AB800080235B029946CA443F04280C3F0C2D04E5
:10AB9000ED19270C2404240C0300200050437A43B1
:10ABA00091463A0053440593030C9A464A43614345
:10ABB00049445144AB44894503D980235B029946FB
:10ABC0004A4400040B0C000C0904091820009946A3
:10ABD000434670435C437E435F43030C9846A4198D
:10ABE00044444A440397A64204D980235B02984612
:10ABF000474403972304029E9A46059B5E44984669
:10AC0000AE42AD4176188E4289410004000C50449A
:10AC100040446D424719B846934649428946C34469
:10AC2000D94498428041A845AD4193459241894518
:10AC300089416D4240422843240C524249420A4312
:10AC4000039B00198018C7184B46DC0D049B750246
:10AC50001D436A1E95414B46F60D7F0235435A024D
:10AC60003C431543FB0100D41CE101216A080D405F
:10AC70001543E207154364084F496144002900DC8D
:10AC8000B0E06B0709D00F222A40042A05D02A1D04
:10AC9000AA42AD416D4264191500E30104D580213B
:10ACA000464AC90014406144454A914200DD26E706
:10ACB0006207ED08640249051543240B4A0D10E7AD
:10ACC0005246324300D17FE0002E00D1DCE030005C
:10ACD00000F096FD02000B3A1D2301009B1A52461C
:10ACE0000839DA408E40164352468A40009B354967
:10ACF000181A03008C46634400200093D3E6250015
:10AD000005434AD0002C00D1B0E0200000F078FDCF
:10AD1000010002000B391D2310005B1A31003500C1
:10AD200008388440D94085400C432648831A009354
:10AD3000002399469B4697E60500254326D1082225
:10AD400000930223002491469B468DE65246009BC9
:10AD5000324310D1154900268C466344494600937E
:10AD600002231943894602209DE65B460197022B88
:10AD700000D0ADE6C3E60D4A0320944663444A463C
:10AD8000009303231A43914652468CE60C2200930B
:10AD90000323050091469B4666E60423994600235B
:10ADA0000093013300249B465EE6C046FF07000087
:10ADB00001FCFFFFB0C80000FF030000FFFFFFFE23
:10ADC000FE0700000DFCFFFF494601231943894699
:10ADD0000026012067E6002380240025434A0193D2
:10ADE00024037EE60120401A382800DD76E61F287D
:10ADF0005BDD1F2223005242511ACB40190020284C
:10AE000003D03B4A6244944025436A1E95412A0080
:10AE10000A4307210D000024154011425BD00F2189
:10AE200000241140042953D0111D914292415242F5
:10AE3000A4180A0023024BD501220024002550E665
:10AE400080231B031C4209D01E4207D133431C033D
:10AE500043461500240B254A019342E68022120343
:10AE600014432403214A240B01973AE600F0C8FC5E
:10AE700001000200153120321C2900DC4BE73400B0
:10AE800008380025844050E700F0BAFC03001A009F
:10AE9000153220301C2A00DC1EE75646083B0022F3
:10AEA0009E4023E7009B9C46E6E61249220061444F
:10AEB0002E008D408A40C640691E8D4132432A4390
:10AEC000C4405307B6D00F2111400429ACD1B1E7DB
:10AED00065076402240BD2081543002201E6802294
:10AEE000120314432403014A240BFAE5FF07000070
:10AEF0003E0400001E040000F8B557464E46454685
:10AF0000DE46E0B51E0017004A000B03520D5B0A37
:10AF10009046420F1A43CD0FCD4C3103C3009446E7
:10AF200070007A0F490AFF009A46B946400DF60FA5
:10AF30001143A04200D1B1E001225640B346B542D0
:10AF400000D188E04246121A002A00DCAEE0002858
:10AF500000D1C1E0BE48804500D151E1802000040D
:10AF60000143382A00DD7BE11F2A00DDEEE12020CD
:10AF70003E00801A0C00D640D14087406246844093
:10AF8000521A781E8741944634432743DC1BA34260
:10AF90009B4162465B42D31A99464B461B0200D442
:10AFA00018E14B465802430A99464B46002B00D104
:10AFB00037E1484600F024FC010008392023220034
:10AFC00048465B1ADA4088408C4043461043884527
:10AFD00000DD36E1C91A4B1C1F2B00DDEAE0202200
:10AFE0002600D21A01009440DE40D8400023914050
:10AFF000621E94418146984631430C43630709D051
:10B000000F232340042B05D0231DA342A4416442F7
:10B01000A1441C004B461B0200D4DEE041468C4B91
:10B020000131994200D1E7E04B468A48E4080340E9
:10B03000180049055B07400223434A0D040B120523
:10B04000ED0722432A4318001100F0BCBB46B2466C
:10B05000A946A046F8BD4246121A002A52DD002831
:10B0600000D19CE0A04500D1CAE08020000401434B
:10B07000382A00DD49E11F2A00DC97E110000E00AC
:10B080002038C640202A04D04020821A91400F4325
:10B09000B9464C46621E944134433AE10A003A43B1
:10B0A00028D0B346B5422BD06B4A4244002A5DD02B
:10B0B00042464446821A002C00D0F5E065461D4306
:10B0C00000D19CE1551E012A00D1FBE1604CA24257
:10B0D00000D1BDE12A00F0E00800384300D1C3E010
:10B0E000501E012A00D1A8E1594CA24200D187E0AC
:10B0F000020036E701225640B346B54200D021E7B0
:10B10000554A4244002A00D1B5E042464446821ADC
:10B11000002C00D138E14E4EB04200D1DEE1802655
:10B12000644636043443A446382A00DD96E11F2ADB
:10B1300000DD24E22026B41AA24664465646B440F6
:10B14000A1461C004E46D440264334005646B34028
:10B150005E1EB3411C436346D340C918E419BC4288
:10B16000BF417F42B94680468944D8E040463B4CC7
:10B170000130204200D0B4E04046002800D044E135
:10B180006046184300D190E10800384300D0AAE19E
:10B190006146DB0849070B436146CC0827E00800FD
:10B1A000384361D0501E012A00D139E1A24227D094
:10B1B00002005DE702001F39CA401100202B03D0B6
:10B1C0004022D31A98400443631E9C4100239946B1
:10B1D00098460C43630700D012E74B464A46E40802
:10B1E0005B072343D408424619498A420ED0240300
:10B1F0005205240B520D22E70A00002400231EE70B
:10B20000DB086246520713436246D4081A00224301
:10B2100000D1FCE180221203144324030C4A240BC6
:10B220000DE7200000F0ECFA010018311F2900DCC6
:10B23000C4E608388440434620000024884500DCEA
:10B24000C8E6044A5B1A104098468146D6E6C046D6
:10B25000FF070000FFFF7FFF01F8FFFFFE07000070
:10B260000F437A1E974191E66146DB0849070B437D
:10B270006146CC08B8E74046D34C0130204200D0AC
:10B28000A2E04046002800D001E16046184300D10A
:10B290005EE10800384300D05FE16146DB08490702
:10B2A0000B436146CC08A2E7C84DA84200D1CFE0CD
:10B2B000802564462D042C43A446382A56DC1F2AD8
:10B2C00000DDD1E020251E00AD1A6446AB40AC4045
:10B2D000D6405D1EAB41344323436446D440091B32
:10B2E00049E06046DC1B461AA34280414042814649
:10B2F00030004E46801B8146000276D44B462343E5
:10B3000000D052E60024002571E739430C00621E8C
:10B310009441E4189C429B415B42634499464B46EE
:10B320001B0200D456E701239C46A84BE0449845F5
:10B3300038D04B46A6480122034018006308144049
:10B340001C43C3071C434308994657E610000E00F0
:10B350002038C640202A04D04020821A91400F4352
:10B36000B9464F467A1E974137430FE662461A4365
:10B3700013005A1E9341FC1AA742BF417F42CB1BC8
:10B3800099465D46804608E666461E4300D1BEE00B
:10B39000561E012A00D109E18C4CA24200D119E1CC
:10B3A0003200C1E642460024002348E620200C007B
:10B3B000801A3E0087408440D640781E8741D140A5
:10B3C00034433C438C44A4E7804A904200D1E9E0F6
:10B3D000DF199F429B4161445B42C918CC077F083B
:10B3E0004B08994680463C43F4E6FC1AA742BF410D
:10B3F00063467F42C91ACB1B99465D46D5E5FF08D7
:10B400004B075D463B43CC08EEE662461A4300D04C
:10B4100082E00B003B431BD1802400252403F9E686
:10B42000DC199C429B41614489465B4299444B46EE
:10B430001B0244D401239846CCE6DC1B6246A3429F
:10B440009B41511A5B42CB1A994601239846A4E5C9
:10B45000FF084B075D463B43CC08D7E662461A43DC
:10B460001400631E9C4179E615006446203DEC40C3
:10B47000A046202A05D040256446AA1A94402343BA
:10B480009A465446631E9C414346234373E76246F3
:10B490001A4323D00A003A4300D0A0E06246DB08FA
:10B4A000520713436246D408B0E60B003B4300D179
:10B4B00028E7FF084B075D463B43CC0897E602238D
:10B4C000984636E7FC1AA742BF4163467F42C91A35
:10B4D000CB1B994601235D4698465EE54B07FF0866
:10B4E0003B43CC0892E6DC1B6046A342B641401ABF
:10B4F0007642801B8146000260D5FC1AA742BF41FC
:10B5000063467F42C91ACB1B99465D4676E5FF0824
:10B510004B073B43CC0867E60A00DB083A4300D1FF
:10B520006FE66246520713436246D4088022120334
:10B53000144207D0C808104204D15D460400FB083D
:10B5400049070B435A0FDB00DB08520713435DE644
:10B550004B07FF083B43CC0849E6DC199C429B4162
:10B56000614489465B4299444B461B0200D431E654
:10B570004A46174B1A400123914698462AE6160080
:10B580006446203EF440A046202A05D0402664466A
:10B59000B21A944023439A465446631E9C41434644
:10B5A0001C43DBE502000024002348E5DC19BC4213
:10B5B000BF41614489467F42B94438E74B46234343
:10B5C00000D19FE606E6C046FE070000FF07000028
:10B5D000FFFF7FFFFF084B073B43CC0816E66246A0
:10B5E000DB08520713436246D40880221203144238
:10B5F00007D0C808104204D15D460400FB08490783
:10B600000B435A0FDB005207DB081343FEE5002310
:10B61000014A1C0013E5C046FF07000070B5050095
:10B620000C481C0316005B000A034900120B490D6D
:10B63000240B5B0D814208D0064A0020934203D1BF
:10B6400020003043431E984170BD01202A43FBD1A6
:10B65000F2E7C046FF0700000A0030B5134C530064
:10B6600009030500090B00205B0DD20FA34204DD86
:10B670000F48834202DD0F4BD01830BD80204003BD
:10B6800001430D48C01A1F2808DD0C48C31AD940D1
:10B690000B005842002AF0D11800EEE7084CC540D4
:10B6A000A446634499400B002B43F2E7FE030000DD
:10B6B0001D040000FFFFFF7F33040000130400009F
:10B6C000EDFBFFFF70B5002816D0C317C5185D400D
:10B6D000C40F280000F094F8114A121A0A2816DC48
:10B6E00003002E0015339E400B23181AC540520547
:10B6F0002D032D0B530D03E000240023002500260D
:10B700001B052B43E40723433000190070BD0B38A1
:10B71000854052052D0300262D0B530DF0E7C04642
:10B720001E04000010B5041E10D000F069F80F4B85
:10B730001B1A0A2811DC0B222100121AD1401530E5
:10B740000A035B058440120B5B0D01E0002300221D
:10B750001B0513432000190010BD22000B38824046
:10B760005B0512030024120B5B0DF1E71E040000C1
:10B7700070B543004602C40FFE201B0E591C750A0B
:10B7800008420CD0E022920094466D07360B6344C9
:10B790001B053343E40723432800190070BD002B29
:10B7A00014D1002D1BD0280000F02AF80A281CDC38
:10B7B0000B232E001B1ADE40030015339D400E4A5A
:10B7C0003603121A5205360B530DE1E7002D09D04E
:10B7D0008022360B1203094B6D071643D8E700236E
:10B7E0000026D5E70026054BD2E703000B3B9D4022
:10B7F0002E000025E3E7C04689030000FF07000094
:10B800001C2101231B04984201D3000C10391B0A90
:10B81000984201D3000A08391B09984201D3000954
:10B82000043902A2105C40187047C04604030202AB
:10B8300001010101000000000000000010B5002916
:10B8400003D1FFF7DDFF203002E00800FFF7D8FF4B
:10B8500010BDC046F0B557464E464546DE46E0B5FB
:10B860000F001900002306009846100083B0002F37
:10B8700007DA33003C0000275E42A74101235B4208
:10B880009846002907DA4346DB430C00984603003C
:10B8900000215842A14134003D0082468946B94208
:10B8A0006AD867D049465046FFF7C8FF834639003B
:10B8B0003000FFF7C3FF5B461B1A9C46203B9B46AC
:10B8C0006BD458465146814060460B00514681403A
:10B8D0000A00BB4200D972E0BB4200D179E03400DB
:10B8E0003D005946A41A9D41002900DA74E0002168
:10B8F000002001260090019159468E400196614634
:10B9000001268E406146009600295FD0D90756086F
:10B910000E435F086146012200230CE0AF4201D1D3
:10B92000A6420AD8A41BBD4124196D410139A418AF
:10B930005D41002906D0AF42F0D9013924196D418B
:10B940000029F8D1009801995B4600196941002B44
:10B950004DDB2E002C00DE406346DC405B46002BB6
:10B9600055DB34009C4023006446A6403200801A18
:10B97000994103E0B04295D9002000214346002BB5
:10B9800004D003000C0000215842A14103B0F0BCD8
:10B99000BB46B246A946A046F0BD624648462023B3
:10B9A000514690409B1AD94003000091009960468F
:10B9B0000B43514681400A00BB4200D88CE700216E
:10B9C000002000900191614600299FD100980199C3
:10B9D000D4E7B142F3D882E7614620260127761AE0
:10B9E00000200021F74000900191019787E762460F
:10B9F00020239B1A2A009A40260013006246D64054
:10BA00002C001E436346DC405B46002BA9DA6246ED
:10BA10002023350094409B1ADD4023002B43A3E7ED
:10BA2000014B18687047C046A801001070B50400AB
:10BA3000830716D102680E4B0E4DD31893432B4249
:10BA40000FD142680A4B0430D31893432B4208D1DC
:10BA50004268074B0430D31893432B42F1D000E0E7
:10BA600001300378002BFBD1FDF701F9200070BDF8
:10BA7000FFFEFEFE8080808003274B00070809043C
:10BA8000050600355C365D1D6B002D2D2D005155D2
:10BA900049544E45572020202020434F5059474CB1
:10BAA000554548455820004241545420202020202C
:10BAB0002020204431202044322020546F6666002C
:10BAC00044476574544765742020202044536574AE
:10BAD00054536574202020200051554954202020C3
:10BAE00020202020202D2E2D2020202020484558A9
:10BAF0002000504C4558464C45585241582054540B
:10BB00004F5052554C455445582000454449540027
:10BB100053415645004C4F414400515549545341FF
:10BB200056454C4F41444353542053495A45484588
:10BB3000582000630067004700566D004E410052D8
:10BB4000696E66006800504849300061300052005C
:10BB50004600740061746D0065707330005A3000E7
:10BB60006D55007265006D65006D6E0047300067B1
:10BB7000616D70004331004332000000000000009E
:10BB8000F7E0C08000030000000003000000000395
:10BB9000000000030000000F00000003000000038D
:10BBA00000000300000300B8ABE80003000003003E
:10BBB00000030003000F000000000000000088AB3D
:10BBC000F8000000000000000F0000000000E0236B
:10BBD000F800000000000F00000000E8ABB8000013
:10BBE00000000F000000F8AB380000000F0000C09C
:10BBF00083F800000000F8ABF800000000E0ABF8AC
:10BC00000080C0E0EF07030100C000000000C0009A
:10BC1000000000C0000000C0000000F0000000C0F4
:10BC2000000000C00000C00000C00017D51D00C00B
:10BC30000000C00000C000C000F0000000000000D4
:10BC4000000015D51F00000000000000F0000000FB
:10BC500000001CC41F0000000000F0000000001DD8
:10BC6000D51700000000F00000001FD507000000FD
:10BC7000F0000018D01F000000001FD51F000000BA
:10BC8000001CD51F0001030703040500010200008A
:10BC9000000000000000F87F000000000000F87FB6
:10BCA000D9110000BD110000A11100008511000094
:10BCB000691100004D110000311100002511000034
:10BCC0001B11000011110000ED100000351E0000D6
:10BCD000690D0000D11B0000410E0000D10E0000D4
:10BCE000691B00009D0F000045070000412900006E
:10BCF000E3110000252900003D280000BD0D0000D3
:10BD00005D0200005D020000812B0000412B00005D
:10BD1000DD2A00003503000069030000D51C000087
:10BD2000BD1A0000591700005D0200008D020000DE
:10BD3000AD0200007D0F000035080000B5270000AF
:10BD400025040000951600006D1600005116000035
:10BD50002916000011160000F5150000D915000085
:10BD6000BD1500005D020000011C0000311500003F
:10BD7000510F0000F51A000089070000210F000094
:10BD80005D020000011500005D0200005D02000080
:10BD90005D0200005D0200005D0200005D02000027
:10BDA000F90200005D020000E1280000DD2500002E
:10BDB0005D020000790300005D0200005D020000EA
:10BDC0005D0200005D020000CD020000AD02000037
:10BDD000DD1B00005D020000DD0E00003D040000E0
:10BDE000751400004D140000311400000914000007
:10BDF000F1130000D5130000B91300009D130000DB
:10BE0000D9290000511D00007D1500008D2900007A
:10BE100025130000D5120000A9120000D907000068
:10BE200025080000010F00001927000099270000D5
:10BE3000452400002D1D00005D02000011030000DC
:10BE4000292A00008D2A0000BD2A0000B503000049
:10BE500091030000211D00005D020000CD030000E1
:10BE60005D0200008D020000CD020000951200006E
:10BE70005D020000000000000000002F000000072D
:10BE8000000700147F147F142E2A7F2A3A231308F8
:10BE900064623649552250000B070000001C224105
:10BEA000000041221C0014083E081408083E08083F
:10BEB00000583800000808080808006060000020EA
:10BEC000100804027F4141417F40427F4040794950
:10BED00049494F414949497F0F08087F084F49495F
:10BEE00049797F49494978030101017F7F494949DF
:10BEF0007F0F4949497F0036360000005B3B000058
:10BF000008142241001414141414004122140803CC
:10BF10000159090F7B4979417F7F0909097F7F49D1
:10BF2000494F787F414141407F4141633E7F4949CC
:10BF300049417F090909017F414949797F0808087A
:10BF40007F41417F4141604141417F7F08080F7837
:10BF50007F404040407F010F017F7F0204087F7FC8
:10BF60004141417F7F0909090F7F4171417F7F096D
:10BF700009794F6F4949497B01017F01017F4040A9
:10BF8000407F1F2040201F7F4078407F63140814AB
:10BF9000634F4878484F6151494543007F41410014
:10BFA00002040810200041417F0004020102044005
:10BFB000404040402227227222705454547C7F44D7
:10BFC00044447C7C444444407C4444447F7C5454FA
:10BFD000541C00047F05011C5454547C7F04040449
:10BFE0007C40447D40406040447D007F10101C70C8
:10BFF000007F4040007C041C047C7C0404047C7CA6
:10C000004444447C7C2424243C3C2424247C7C0420
:10C0100004040C5C5454547400047F44407C40403D
:10C02000407C047C20100C7C4070407C44247C4884
:10C03000441C5050507C4464544C44087F4141009F
:10C0400000007F00000041417F081C041C101CFF01
:10C05000F7E3C1FF7F415D417F7F5B415F7F7F45AC
:10C0600055517F7F5555417F7F7177417F7F515576
:10C07000457F7F4155457F7F797D417F7F41554198
:10C080007F7F5155417F7F4175417F7F4155417F82
:10C090007F415D5D7F7F415D637F7F4155557F7F40
:10C0A0004175757F7C1514157C705554557C7C1733
:10C0B00015177C745755577C7F097F494974547C08
:10C0C000545C7C4544457C784A484A787C09112177
:10C0D0007C780A0A0A787C4140417C784240427868
:10C0E00060404D48787C444438447F0105273C60DB
:10C0F000584658607C44477D017E50101E10067ED5
:10C10000027E02775D4941637C44447C043E494998
:10C11000493E5F7101715F081C3E080808183F180E
:10C1200008080C7E0C0808083E1C083E060A12226D
:10C1300022120A063E3E30282422222428303E08BD
:10C140001C3E7F00061E7E1E06303C3F3C30007FBA
:10C150003E1C081436773614047E7F7E041C496327
:10C16000491C00227F220010387C101F00070507A1
:10C170000008082A080822140814227F7F49494130
:10C18000007F007F003E283820202030282422080D
:10C190007F01010360407F010344445F44447C7C91
:10C1A00054541C001D1517000404121F1045257D52
:10C1B00049451D5151517D1C221C221C505854527E
:10C1C0005114741C1714515254585000005500005B
:10C1D0004000400040001C141C0000000800000843
:10C1E0004C3E19087E7F7F7F7E7E7B7B7B7E7E73CD
:10C1F00073737E7E6363637E7E4341437E3E222271
:10C20000223E3E3E3E3E3E1C3622361C1C3E3E3EFC
:10C210001C74465F467477415D41777C7E0F7E7C5F
:10C2200055015501551E5272521E3E2E3E3A3E0396
:10C23000417F41037E435A437E3E636F6B3E6355AD
:10C240004955637E4E4A4A7C386C7F7C382A202AC6
:10C25000202A5555005555084C7F4C083E632263F3
:10C260003E1F047C141C005F557D0023434843237C
:10C270003E003E2A3A7830180C0667415C416778E8
:10C2800000784B7B221D1813231E1914241F1A1526
:10C2900025201B1626211C1712121110000104075D
:10C2A0000A0205080B0306090C0D0E0F0007000813
:10C2B000000A010002070208020100030109030449
:10C2C00002040205030500063031323334353637B7
:10C2D00038392EA42B2DBAB9C1BBB7BFC2EFA9C440
:10C2E000AA68534354B2D9A860A7CF6667E3E300B6
:10C2F0000000004A78DEB14105A3923A019D234037
:10C30000CC8AEDFF9E58D23D0F4BC25D8A41973FCC
:10C3100017C557CA85E1DF44E15D2E7244EE6441E2
:10C32000113102DE0B860B3913A630A819A0E23CAE
:10C33000A356F5D48117CD3D7C645ED5E6B0303B85
:10C34000C43F883E01A12040A60F5D50558EF740A6
:10C35000666666666612714000000000D0BCF84058
:10C3600053160C29DAA4073C346620F17678A33DF5
:10C37000E441CB0F3715B53E1C7E625DAF8B774035
:10C38000AF6AED78F771603A153F4F5EBA61E93CEC
:10C39000EDB7B6C8DC79B239C5A2EAB19990603A76
:10C3A00089C029197296603A8533E91183D82D3AEC
:10C3B000A427278E556C263B668B3F09A102793A4C
:10C3C0006FBE9CB1FD7226BB04D1B3316476913A45
:10C3D0002A52A35F40EC87BA16B2073C66CBABBAD1
:10C3E0009DD21E2AD4E37D3FCCC068A24D716E3E23
:10C3F00036DA19C20BFE1E40AE47E11621E4AF410A
:10C40000968B4CCC59F6BA3C6EF0A2A255778D3F74
:10C4100033BB000035BB000037BB000039BB000058
:10C420003CBB00003FBB000044BB000046BB00001B
:10C430004BBB000088BA00004EBB000050BB0000A0
:10C4400052BB000054BB000067BB000058BB00009B
:10C45000000000105DBB000060BB000063BB00007B
:10C4600066BB000071BB000069BB00000200001049
:10C4700005000010080000100B0000100E00001056
:10C480001100001014000010170000101900001017
:10C490006CBB00006FBB000074BB000077BB0000EA
:10C4A000290300007D020000E9020000A90300004A
:10C4B000510400005D0400002D1800000D1800005C
:10C4C00075120000790C00005D0200005D020000A2
:10C4D00089330000193400005D0200007934000047
:10C4E0003D0C00005D020000ED040000DD190000BD
:10C4F000E9020000D1040000990600005D0200007E
:10C50000D5210000B92100009D21000081210000FB
:10C5100065210000492100002D210000212100009B
:10C52000172100000D210000D11F0000910900001B
:10C530006D09000085090000091F00003D09000089
:10C5400025090000591F0000ED08000069050000E2
:10C550005D02000085050000A50500005D020000E9
:10C560005D020000000000004FBB610567ACDD3FCD
:10C57000182D4454FB21E93F9BF681D20B73EF3F0A
:10C58000182D4454FB21F93FE2652F227F2B7A3C82
:10C59000075C143326A6813CBDCBF07A8807703C3B
:10C5A000075C143326A6913C000000000000000048
:10C5B000000000000000E03F000000000000E0BFBD
:10C5C0000000E0FE422EE63F0000E0FE422EE6BF05
:10C5D000763C7935EF39EA3D763C7935EF39EABD7D
:10C5E000FB21F93FFB2109407CD91240FB21194076
:10C5F0007A6A1F407CD92240BBFD2540FB2129409F
:10C600003A462C407A6A2F405C4731407CD9324010
:10C610009C6B3440BBFD3540DB8F3740FB213940FC
:10C620001BB43A403A463C405AD83D407A6A3F40B3
:10C630004C7E40405C4741406C1042407CD94240B7
:10C640008CA243409C6B4440AC344540BBFD45400C
:10C65000CBC64640DB8F4740EB584840FB21494062
:10C6600083F9A200444E6E00FC291500D157270023
:10C67000DD34F50062DBC0003C9995004190430039
:10C680006351FE00BBDEAB00B761C5003A6E24000B
:10C69000D24D42004906E00009EA2E001C92D1006A
:10C6A000EB1DFE0029B11C00E83EA700F535820015
:10C6B00044BB2E009CE98400B4267000417E5F00DC
:10C6C000D6913900538339009CF439008B5F840084
:10C6D00028F9BD00F81F3B00DEFF97000F9805000A
:10C6E000112FEF000A5A8B006D1F6D00CF7E3600B0
:10C6F00009CB2700464FB7009E663F002DEA5F003A
:10C70000BA277500E5EBC7003D7BF100F73907005C
:10C7100092528A00FB6BEA001FB15F00085D8D003A
:10C72000300356007BFC4600F0AB6B0020BCCF0012
:10C7300036F49A00E3A91D005E619100081BE60033
:10C7400085996500A0145F008D40680080D8FF00C7
:10C7500027734D0006063100CA561500C9A873009C
:10C760007BE260006B8CC00000000040FB21F93FC1
:10C77000000000002D44743E000000809846F83C04
:10C780000000006051CC783B00000080831BF03932
:10C790000000004020257A38000000802282E33625
:10C7A000000000001DF369350200000003000000D6
:10C7B00004000000060000002024282C383C4044DF
:10C7C000484C0207020802010003010903040204A5
:10C7D0000205030500063F0025730D0A0D0A00251A
:10C7E000730D0A00444D5F53444B3E20000000008F
:10C7F000AC9A0000389A0000949900004C9900000F
:10C8000094990000749A0000949900004C990000DB
:10C81000389A0000389A0000749A00004C99000081
:10C82000529900005299000052990000829A00002B
:10C83000389A0000389A0000949900004899000046
:10C8400094990000749A000094990000489900009F
:10C85000389A0000389A0000749A00004899000045
:10C860005299000052990000529900007E9A0000EF
:10C87000F8A20000E6A20000C4A20000EEA20000A0
:10C88000C4A20000C6A50000C4A20000EEA20000E1
:10C89000E6A20000E6A20000C6A50000EEA200008D
:10C8A000B0A20000B0A20000B0A200003CA60000B0
:10C8B00006AB0000C4AA0000C4AA0000C0AA000081
:10C8C000CAAA0000CAAA0000D6AD0000C0AA000093
:10C8D000CAAA0000D6AD0000CAAA0000C0AA000083
:10C8E0006AAD00006AAD00006AAD000040AE000015
:08C8F00064EFFF7F010000006E
:10C8F800A1006DA100A14200A14E00A16500A17098
:10C9080000A16E00A1A1009D00A40001010000008B
:10C9180001013C2D0000002D0000002D0000002D1D
:10C928000000002D0000002D000000FF00000000A6
:10C9380000000000000000000000000000000000EF
:10C9480000000000000000000000000000000000DF
:10C95800000000000000000000000000002D0000A2
:10C96800002D0000002D0000002D0000002D00000B
:10C97800002D0000000A0000000000000000000078
:10C98800000000000000000000000000000000009F
:10C99800000000000000000000000000000000008F
:10C9A800000000000000000000000000000000007F
:10C9B800000000000000000000000000000000006F
:10C9C800000000000000000000000000000000005F
:10C9D800000000000000000000000000000000004F
:10C9E800000000000000000000000000000000003F
:10C9F800000000000000000000000000000000002F
:10CA0800000000000000000000000000000000001E
:10CA1800000000000000000000000000000000000E
:10CA280000000000000000000000000000000000FE
:10CA380000000000000000000000000000000000EE
:10CA480000000000000000000000000000000000DE
:10CA580000000000000000000000000000000000CE
:10CA680000000000000000000000000000000000BE
:10CA780000000000002D0000002D0000002D000027
:10CA8800002D0000002D0000002D00000005000012
:10CA9800FFFFFFFF4D000000B00100100000000084
:10CAA800000000009C040010040500106C05001034
:10CAB800000000000000000000000000000000006E
:10CAC800000000000000000000000000000000005E
:10CAD800000000000000000000000000000000004E
:10CAE800000000000000000000000000000000003E
:10CAF800000000000000000000000000000000002E
:10CB0800000000000000000000000000000000001D
:10CB1800000000000000000000000000000000000D
:10CB280000000000000000000000000000000000FD
:10CB380000000000000000000000000000000000ED
:10CB480000000000000000000100000000000000DC
:10CB58000E33CDAB34126DE6ECDE05000B000000A1
:10CB680000000000000000000000000000000000BD
:10CB780000000000000000000000000000000000AD
:10CB8800000000000000000000000000000000009D
:10CB9800000000000000000000000000000000008D
:040000030000902148
:00000001FF
